:020000040000FA
:0408000055EF0BF0B5
:1008100003B272EF05F0F2B490EF05F09EB098EFDE
:1008200005F09EB2A0EF05F0F2A81AEF04F0F2B2C4
:1008300021EF04F0F2B01FEF04F004EF0BF0F2969A
:10084000F290CD90F2929EA02BEF04F00101533F65
:100850002BEF04F0542BAEC1B2F1AFC1B3F1B0C174
:10086000B4F1B1C1B5F1AAC1AEF1ABC1AFF1ACC148
:10087000B0F1ADC1B1F1A6C1AAF1A7C1ABF1A8C158
:10088000ACF1A9C1ADF1A2C1A6F1A3C1A7F1A4C168
:10089000A8F1A5C1A9F19EC1A2F19FC1A3F1A0C178
:1008A000A4F1A1C1A5F19AC19EF19BC19FF19CC188
:1008B000A0F19DC1A1F196C19AF197C19BF198C198
:1008C0009CF199C19DF1CECF96F1CFCF97F153C155
:1008D00098F154C199F1CF6ACE6A0101536B546B00
:1008E0009E90CD800FBC0F8E0FBA7AEF04F00F8A66
:1008F00004EF0BF00F8C0FBEB6EF04F096C19AF127
:1009000097C19BF198C19CF199C19DF19AC19EF14B
:100910009BC19FF19CC1A0F19DC1A1F19EC1A2F11B
:100920009FC1A3F1A0C1A4F1A1C1A5F1A2C1A6F1EB
:10093000A3C1A7F1A4C1A8F1A5C1A9F1A6C1AAF1BB
:10094000A7C1ABF1A8C1ACF1A9C1ADF1AAC1AEF18B
:10095000ABC1AFF1ACC1B0F1ADC1B1F1AEC1B2F15B
:10096000AFC1B3F1B0C1B4F1B1C1B5F101015E6B7A
:100970005F6B606B616B96515E2797515F23985157
:100980006023995161239A515E279B515F239C51AB
:1009900060239D5161239E515E279F515F23A0518B
:1009A0006023A1516123A2515E27A3515F23A4516B
:1009B0006023A5516123A6515E27A7515F23A8514B
:1009C0006023A9516123AA515E27AB515F23AC512B
:1009D0006023AD516123AE515E27AF515F23B0510B
:1009E0006023B1516123B2515E27B3515F23B451EB
:1009F0006023B5516123D8900101613360335F33C7
:100A00005E33D8900101613360335F335E33D89039
:100A10000101613360335F335E3300C10CF101C10A
:100A20000DF102C10EF103C10FF104C110F105C1B6
:100A300011F106C112F107C113F108C114F109C186
:100A400015F10AC116F10BC117F134C135F111B816
:100A500035EF05F00101620E046F010E056F000E07
:100A6000066F000E076F3EEF05F00101A70E046F41
:100A7000020E056F000E066F000E076F5EC100F1DB
:100A80005FC101F160C102F161C103F134EC2CF0EE
:100A900003BF04D019BE02D019A0108C11A056EFCC
:100AA00005F010BA56EF05F00F80108A0CC100F166
:100AB0000DC101F10EC102F10FC103F110C104F12A
:100AC00011C105F112C106F113C107F114C108F1FA
:100AD00015C109F116C10AF117C10BF135C134F185
:100AE00004EF0BF00392ABB2AB98AB88030103EEBB
:100AF00000F080517F0BE92604C0EFFF802B81516D
:100B0000805D700BD8A48B8200008051815D700BDA
:100B1000D8A48B9281518019D8B4079004EF0BF0C0
:100B2000F2940101453F04EF0BF0462B04EF0BF06C
:100B30009E900101533F04EF0BF0542B04EF0BF098
:100B40009E9211B823EF08F0040066A1A8EF05F00B
:100B50008BB4B2EF05F010ACB2EF05F08B84109CB3
:100B6000B3EF05F08B94077C07ACCEEF05F0C274B1
:100B7000C2B4C8EF05F0C3CFB7F5C4CFB8F50501CF
:100B8000D890B833B733D890B833B733CFEF05F038
:100B9000C3CF55F1C4CF56F1CFEF05F0C28207B4F1
:100BA0003CEF06F047C14BF148C14CF149C14DF152
:100BB0004AC14EF15EC162F15FC163F160C164F18F
:100BC00061C165F196C1B6F197C1B7F198C1B8F1AD
:100BD00099C1B9F19AC1BAF19BC1BBF19CC1BCF1F9
:100BE0009DC1BDF19EC1BEF19FC1BFF1A0C1C0F1C9
:100BF000A1C1C1F1A2C1C2F1A3C1C3F1A4C1C4F199
:100C0000A5C1C5F1A6C1C6F1A7C1C7F1A8C1C8F168
:100C1000A9C1C9F1AAC1CAF1ABC1CBF1ACC1CCF138
:100C2000ADC1CDF1AEC1CEF1AFC1CFF1B0C1D0F108
:100C3000B1C1D1F1B2C1D2F1B3C1D3F1B4C1D4F1D8
:100C4000B5C1D5F1B7C5B9F5B8C5BAF5B9C5BBF5E4
:100C5000BAC5BCF5010155515B2756515C23E86AC2
:100C60005D230E2E3CEF06F05CC157F15DC158F1DB
:100C70005B6B5C6B5D6B078E0201002F04EF0BF06A
:100C80003C0E006F1A50E00BE00AE866128818BEAE
:100C900002D018B4108E00C10CF101C10DF102C1D7
:100CA0000EF103C10FF104C110F105C111F106C12C
:100CB00012F107C113F108C114F109C115F10AC1FC
:100CC00016F10BC117F134C135F181AA1CEF07F001
:100CD00030A0EDEF06F005012F51000AD8B41CEF4B
:100CE00007F005012F51010AD8B4A6EF06F005015F
:100CF0002F51020AD8B4E7EF06F005012F51030A7D
:100D0000D8B4E7EF06F005012F51040AD8B4E7EF95
:100D100006F005012F51050AD8B4E7EF06F00501EA
:100D20002F51060AD8B4E7EF06F005012F51070A44
:100D3000D8B4E7EF06F005012F51320AD8B4A4EF7A
:100D400006F02F6B1CEF07F01CEF07F0050157674B
:100D5000B1EF06F05867B1EF06F05967B1EF06F052
:100D60005A67B5EF06F01CEF07F05BC500F15CC5F4
:100D700001F15DC502F15EC503F10101010E046FD1
:100D8000000E056F000E066F000E076F34EC2CF09E
:100D900000C15BF501C15CF502C15DF503C15EF503
:100DA0000067DAEF06F00167DAEF06F00267DAEFC4
:100DB00006F003671CEF07F057C55BF558C55CF5F7
:100DC00059C55DF55AC55EF50F881CEF07F00501A2
:100DD0003067EDEF06F01CEF07F00FBE02EF07F0F3
:100DE00010A007EF07F001014767FEEF06F0486724
:100DF000FEEF06F04967FEEF06F04A6702EF07F0E4
:100E000007EF07F007AE07EF07F019EF07F005014E
:100E1000312F1CEF07F03C0E316F302F1CEF07F025
:100E20000101000E626FE00E636FA50E646F010E8C
:100E3000656F0501306B0F880501666B37B722EFD0
:100E400007F066810CC100F10DC101F10EC102F184
:100E50000FC103F110C104F111C105F112C106F176
:100E600013C107F114C108F115C109F116C10AF146
:100E700017C10BF135C134F100C10CF101C10DF105
:100E800002C10EF103C10FF104C110F105C111F14E
:100E900006C112F107C113F108C114F109C115F11E
:100EA0000AC116F10BC117F134C135F101018A678E
:100EB00061EF07F08B6761EF07F08C6761EF07F078
:100EC0008D6765EF07F095EF07F08EC100F18FC1D8
:100ED00001F190C102F191C103F10101010E046F12
:100EE000000E056F000E066F000E076F34EC2CF03D
:100EF00000C18EF101C18FF102C190F103C191F1E6
:100F000000678AEF07F001678AEF07F002678AEF50
:100F100007F0036795EF07F08AC18EF18BC18FF15F
:100F20008CC190F18DC191F10F80D57ED5BE6DD071
:100F3000D6CF47F1D7CF48F145C149F1E86AE8CFAC
:100F40004AF119BE02D019A0108C109047C100F1CF
:100F500048C101F149C102F14AC103F101010A0E80
:100F6000046F000E056F000E066F000E076F34EC65
:100F70002CF003AF1080010154A7CBEF07F00F9ABC
:100F80000F9C0F9E0101000E5E6F600E5F6F3D0EA5
:100F9000606F080E616F010147BFDBEF07F0486724
:100FA000DBEF07F04967DBEF07F04A67DBEF07F09D
:100FB000F28800EF08F0F2985E6B5F6B606B616B1C
:100FC000966B976B986B996B9A6B9B6B9C6B9D6BFD
:100FD0009E6B9F6BA06BA16BA26BA36BA46BA56BAD
:100FE000A66BA76BA86BA96BAA6BAB6BAC6BAD6B5D
:100FF000AE6BAF6BB06BB16BB26BB36BB46BB56B0D
:10100000D76AD66A0101456B466B0CC100F10DC170
:1010100001F10EC102F10FC103F110C104F111C1C0
:1010200005F112C106F113C107F114C108F115C190
:1010300009F116C10AF117C10BF135C134F104EF02
:101040000BF004EF0BF00201002F6DEF0AF0D59EBC
:10105000D6CF47F1D7CF48F145C149F1E86AE8CF8B
:101060004AF1D76AD66A0101456B466BD58E1A5094
:10107000E00BE00AE866128818BE02D018B4108EA1
:1010800017AE1C8C00C10CF101C10DF102C10EF1B3
:1010900003C10FF104C110F105C111F106C112F134
:1010A00007C113F108C114F109C115F10AC116F104
:1010B0000BC117F134C135F10FA0109A11B86CEFC4
:1010C00008F00101620E046F010E056F000E066F3D
:1010D000000E076F75EF08F00101A70E046F020EF6
:1010E000056F000E066F000E076F47C100F148C183
:1010F00001F149C102F14AC103F134EC2CF003BF04
:1011000088EF08F019BE02D019A0108C11B00F8022
:101110000CC100F10DC101F10EC102F10FC103F1CB
:1011200010C104F111C105F112C106F113C107F19B
:1011300014C108F115C109F116C10AF117C10BF16B
:1011400035C134F102013C0E006F00C10CF101C148
:101150000DF102C10EF103C10FF104C110F105C17F
:1011600011F106C112F107C113F108C114F109C14F
:1011700015F10AC116F10BC117F134C135F181AA7D
:1011800076EF09F030A047EF09F005012F51000A72
:10119000D8B476EF09F005012F51010AD8B400EF59
:1011A00009F005012F51020AD8B441EF09F00501F9
:1011B0002F51030AD8B441EF09F005012F51040A59
:1011C000D8B441EF09F005012F51050AD8B441EF19
:1011D00009F005012F51060AD8B441EF09F00501C5
:1011E0002F51070AD8B441EF09F005012F51320AF7
:1011F000D8B4FEEF08F02F6B76EF09F076EF09F028
:10120000050157670BEF09F058670BEF09F05967B5
:101210000BEF09F05A670FEF09F076EF09F05BC5A5
:1012200000F15CC501F15DC502F15EC503F101018C
:10123000010E046F000E056F000E066F000E076FA3
:1012400034EC2CF000C15BF501C15CF502C15DF529
:1012500003C15EF5006734EF09F0016734EF09F070
:10126000026734EF09F0036776EF09F057C55BF5C5
:1012700058C55CF559C55DF55AC55EF50F8876EF22
:1012800009F00501306747EF09F076EF09F00FBE6E
:101290005CEF09F010A061EF09F00101476758EF1A
:1012A00009F0486758EF09F0496758EF09F04A67B5
:1012B0005CEF09F061EF09F007AE61EF09F073EF41
:1012C00009F00501312F76EF09F03C0E316F302F18
:1012D00076EF09F00101000E626FE00E636FA50E5C
:1012E000646F010E656F0501306B0F880501666B39
:1012F00037B77CEF09F066810CC100F10DC101F137
:101300000EC102F10FC103F110C104F111C105F1C9
:1013100012C106F113C107F114C108F115C109F199
:1013200016C10AF117C10BF135C134F100C10CF13E
:1013300001C10DF102C10EF103C10FF104C110F1A1
:1013400005C111F106C112F107C113F108C114F171
:1013500009C115F10AC116F10BC117F134C135F1FC
:1013600001018A67BBEF09F08B67BBEF09F08C675F
:10137000BBEF09F08D67BFEF09F0EFEF09F08EC109
:1013800000F18FC101F190C102F191C103F101019E
:10139000010E046F000E056F000E066F000E076F42
:1013A00034EC2CF000C18EF101C18FF102C190F13B
:1013B00003C191F10067E4EF09F00167E4EF09F080
:1013C0000267E4EF09F00367EFEF09F08AC18EF1DD
:1013D0008BC18FF18CC190F18DC191F10F80109074
:1013E00047C100F148C101F149C102F14AC103F10D
:1013F00001010A0E046F000E056F000E066F000E4D
:10140000076F34EC2CF003AF1080010154A715EFE7
:101410000AF00F9A0F9C0F9E0101000E5E6F600E86
:101420005F6F3D0E606F080E616F47C100F148C1EC
:1014300001F149C102F14AC103F10101140E046F27
:10144000050E056F000E066F000E076F34EC2CF0D2
:1014500003AF2EEF0AF0F28853EF0AF0F2985E6BBA
:101460005F6B606B616B966B976B986B996B9A6B0C
:101470009B6B9C6B9D6B9E6B9F6BA06BA16BA26B20
:10148000A36BA46BA56BA66BA76BA86BA96BAA6BD0
:10149000AB6BAC6BAD6BAE6BAF6BB06BB16BB26B80
:1014A000B36BB46BB56B0CC100F10DC101F10EC192
:1014B00002F10FC103F110C104F111C105F112C114
:1014C00006F113C107F114C108F115C109F116C1E4
:1014D0000AF117C10BF135C134F104008BB478EF78
:1014E0000AF010AC78EF0AF08B84109C79EF0AF0C8
:1014F0008B94077C07AC94EF0AF0C274C2B48EEFF1
:101500000AF0C3CFB7F5C4CFB8F50501D890B8330A
:10151000B733D890B833B73395EF0AF0C3CF55F14E
:10152000C4CF56F195EF0AF0C28207B402EF0BF078
:1015300047C14BF148C14CF149C14DF14AC14EF18F
:101540005EC162F15FC163F160C164F161C165F1C7
:1015500096C1B6F197C1B7F198C1B8F199C1B9F187
:101560009AC1BAF19BC1BBF19CC1BCF19DC1BDF157
:101570009EC1BEF19FC1BFF1A0C1C0F1A1C1C1F127
:10158000A2C1C2F1A3C1C3F1A4C1C4F1A5C1C5F1F7
:10159000A6C1C6F1A7C1C7F1A8C1C8F1A9C1C9F1C7
:1015A000AAC1CAF1ABC1CBF1ACC1CCF1ADC1CDF197
:1015B000AEC1CEF1AFC1CFF1B0C1D0F1B1C1D1F167
:1015C000B2C1D2F1B3C1D3F1B4C1D4F1B5C1D5F137
:1015D000B7C5B9F5B8C5BAF5B9C5BBF5BAC5BCF557
:1015E000010155515B2756515C23E86A5D230E2E9D
:1015F00002EF0BF05CC157F15DC158F15B6B5C6BA6
:101600005D6B078E04EF0BF002C0E0FF005001C0DD
:10161000D8FF1000A6B20AEF0BF00CC0A9FF0BC058
:10162000A8FFA69EA69CA684F29E550EA76EAA0EA3
:10163000A76EA682F28EA694A6B21CEF0BF00C2A1F
:101640001200A96EA69EA69CA680A8500C2A120085
:1016500004012C0E826F73EC0EF02FEC2DF00C5069
:1016600021EC0BF0E8CF00F10C5021EC0BF0E8CFAF
:1016700001F101AF41EF0BF00101FF0E026FFF0E10
:10168000036FD2EC2CF029674DEF0BF00401200E14
:10169000826F73EC0EF052EF0BF004012D0E826F8F
:1016A00073EC0EF0DCEC2AF01200306A076A0F6A65
:1016B000106A116A126A136A0F010D0EC16E860E4E
:1016C000C06E030EC26E0F01680E896E130E926E0D
:1016D000080E8A6EF30E936E8B6A900E946EC80E8F
:1016E00021EC0BF0E8CFE8FF1098E8A0108810A8D4
:1016F00005D00E0E226E8E0E236E04D00F0E226EBB
:101700008F0E236EAEEC2DF0F18EF19EFC0E21ECCF
:101710000BF0E8CF0BF00BA011800BA211820BA4F1
:1017200011840BA81188C90E21EC0BF0E8CF17F03B
:10173000CA0E21EC0BF0E8CF18F0CB0E21EC0BF029
:10174000E8CF19F0CC0E21EC0BF0E8CF1AF0CD0E5B
:1017500021EC0BF0E8CF2FF01C6A1D6A0E6A010124
:101760005B6B5C6B5D6B576B586BF29A0101476B5F
:10177000486B496B4A6B4B6B4C6B4D6B4E6B4F6BB5
:10178000506B516B526B456B466BD76AD66A0F0133
:10179000280ED56EF28A9D90B00ECD6E01015E6B63
:1017A0005F6B606B616B626B636B646B656B666BCD
:1017B000676B686B696B536B546BCF6ACE6A0F9A19
:1017C0000F9C0F9E9D80760ECA6E9D8202013C0E7C
:1017D000006FCC6A160E21EC0BF0E8CF00F1170E6B
:1017E00021EC0BF0E8CF01F1180E21EC0BF0E8CF63
:1017F00002F1190E21EC0BF0E8CF03F1010103AF68
:101800001CEF0CF02FEC2DF0160E0C6E00C10BF03F
:101810000AEC0BF0170E0C6E01C10BF00AEC0BF08A
:10182000180E0C6E02C10BF00AEC0BF0190E0C6EC8
:1018300003C10BF00AEC0BF000C18AF101C18BF17E
:1018400002C18CF103C18DF100C18EF101C18FF194
:1018500002C190F103C191F11A0E21EC0BF0E8CF17
:1018600000F11B0E21EC0BF0E8CF01F11C0E21EC76
:101870000BF0E8CF02F11D0E21EC0BF0E8CF03F1E5
:10188000010103AF72EF0CF02FEC2DF01A0E0C6E6D
:1018900000C10BF00AEC0BF01B0E0C6E01C10BF03B
:1018A0000AEC0BF01C0E0C6E02C10BF00AEC0BF0F4
:1018B0001D0E0C6E03C10BF00AEC0BF01A0E21EC9E
:1018C0000BF0E8CF00F11B0E21EC0BF0E8CF01F19B
:1018D0001C0E21EC0BF0E8CF02F11D0E21EC0BF0F9
:1018E000E8CF03F100C192F101C193F102C194F17B
:1018F00003C195F1240EAC6E900EAB6E240EAC6E4F
:10190000080EB86E000EB06E1F0EAF6E0401806B35
:10191000816B0F01900EAB6E0F019D8A0301806BEE
:10192000816BC26B8B9252EC32F052EC32F0B0EC25
:1019300033F031EC30F0200E21EC0BF0E8CF2FF536
:1019400005012F51FF0AD8A4ADEF0CF02F6B200E2C
:101950000C6E2FC50BF00AEC0BF00501010E306F79
:101960003C0E316F250E21EC0BF0E8CF00F1260E76
:1019700021EC0BF0E8CF01F1270E21EC0BF0E8CFC2
:1019800002F1280E21EC0BF0E8CF03F1010103AFC7
:10199000E4EF0CF02FEC2DF0250E0C6E00C10BF0D7
:1019A0000AEC0BF0260E0C6E01C10BF00AEC0BF0EA
:1019B000270E0C6E02C10BF00AEC0BF0280E0C6E19
:1019C00003C10BF00AEC0BF000C157F501C158F54B
:1019D00002C159F503C15AF500C15BF501C15CF5BF
:1019E00002C15DF503C15EF5290E21EC0BF0E8CFD5
:1019F0005FF5050160515F5DD8A05FC560F5210E00
:101A000021EC0BF0E8CF00F1220E21EC0BF0E8CF37
:101A100001F1230E21EC0BF0E8CF02F1240E21ECB2
:101A20000BF0E8CF03F1010103AF45EF0DF02FEC10
:101A30002DF0210E0C6E00C10BF00AEC0BF0220E03
:101A40000C6E01C10BF00AEC0BF0230E0C6E02C100
:101A50000BF00AEC0BF0240E0C6E03C10BF00AEC39
:101A60000BF0210E21EC0BF0E8CF00F1220E21EC5F
:101A70000BF0E8CF01F1230E21EC0BF0E8CF02F1DF
:101A8000240E21EC0BF0E8CF03F100C161F501C198
:101A900062F502C163F503C164F579EC2FF05FECE8
:101AA0002EF0B7EC2DF030A0B6EF0DF005012F5160
:101AB000020A16E005012F51030A19E005012F5112
:101AC000040A24E005012F51050A2BE005012F51DE
:101AD000060A39E005012F51070A3FE0B6EF0DF085
:101AE000602FB3EF0DF05FC560F5B6EF0DF0B0C538
:101AF00000F101010F0E001701010051000A36E04C
:101B000001010051050A32E0B3EF0DF0B0C500F15C
:101B100001010F0E001701010051000A27E0B3EF89
:101B20000DF00501B051000A21E00501B051150A80
:101B30001DE00501B051300A19E00501B051450A18
:101B400015E0B3EF0DF00501B051000A0FE00501FB
:101B5000B051300A0BE0B3EF0DF00501B051000AAF
:101B600005E0B3EF0DF081BAEFEF33F0079000011D
:101B7000F28EF28C12AE03D012BCB2EF18F007B0A6
:101B800062EF29F00FB0FEEF22F010BEFEEF22F060
:101B900012B8FEEF22F00FB89AEF1CF0030180514B
:101BA00081197F0BD8B462EF29F013EE00F0815158
:101BB0007F0BE126812BE7CFE8FFE00BD8B462EF83
:101BC00029F023EE82F0C2513F0BD926E7CFDFFF89
:101BD000C22BDF50780AD8A462EF29F007808EC1AB
:101BE00000F18FC101F190C102F191C103F1010136
:101BF000040E046F000E056F000E066F000E076FD7
:101C000034EC2CF000AF0EEF0EF00101030E8E6FDE
:101C1000000E8F6F000E906F000E916F03018251C6
:101C2000720AD8B4E3EF22F08251520AD8B4E3EF3B
:101C300022F08251750AD8B4E3EF22F08251630A90
:101C4000D8B41CEF26F08251690AD8B492EF1FF085
:101C500082517A0AD8B4A5EF20F08251490AD8B44B
:101C600031EF1FF08251500AD8B44FEF1EF082516D
:101C7000700AD8B492EF1EF08251540AD8B4BDEF66
:101C80001EF08251740AD8B403EF1FF08251410A4A
:101C9000D8B489EF0FF082514B0AD8B487EF0EF019
:101CA00082516D0AD8B4BCEF13F082514D0AD8B4FA
:101CB000D5EF13F08251730AD8B413EF22F082519A
:101CC000530AD8B478EF22F082514C0AD8B464EFAA
:101CD00014F08251590AD8B40DEF13F012AE01D0AE
:101CE000128C53EF26F0040114EE00F080517F0BAC
:101CF000E12682C4E7FF802B120004010D0E826FE3
:101D000073EC0EF00A0E826F73EC0EF012000401F9
:101D10004B0E826F73EC0EF004012C0E826F73EC8D
:101D20000EF081B802D02FB630D003018351430AA0
:101D3000D8B4CCEF0EF003018351630AD8B4CEEFD0
:101D40000EF003018351520AD8B4D0EF0EF0030114
:101D50008351720AD8B4D2EF0EF003018351470ABF
:101D6000D8B4D4EF0EF003018351670AD8B4D6EF8C
:101D70000EF003018351540AD8B4D8EF0EF00301DA
:101D80008351740AD8B447EF0FF003018351550A09
:101D9000D8B4DAEF0EF082D02F807AD02F9078D09E
:101DA0002F8276D02F9274D02F8472D02F9470D03F
:101DB0002F866ED084C330F185C331F186C332F1F2
:101DC00087C333F10101296B7DEC2DF0F4EC2CF08D
:101DD00000C104F101C105F102C106F103C107F11F
:101DE00070EC2DF0200EF86EF76AF66A0900F5CF58
:101DF0002CF10900F5CF2DF10900F5CF2EF10900E6
:101E0000F5CF2FF10900F5CF30F10900F5CF31F111
:101E10000900F5CF32F10900F5CF33F10101296B4B
:101E20007DEC2DF0F4EC2CF034EC2CF0006720EF7E
:101E30000FF0016720EF0FF0026720EF0FF003674C
:101E400001D025D004014E0E826F73EC0EF0040118
:101E50006F0E826F73EC0EF004014D0E826F73EC07
:101E60000EF00401610E826F73EC0EF00401740E2B
:101E7000826F73EC0EF00401630E826F73EC0EF050
:101E80000401680E826F73EC0EF051EF26F02F966E
:101E9000CD0E0C6E2FC00BF00AEC0BF0CD0E21EC2A
:101EA0000BF0E8CF2FF02FB006D00401630E826F45
:101EB00073EC0EF005D00401430E826F73EC0EF04C
:101EC0002FB206D00401720E826F73EC0EF005D0B3
:101ED0000401520E826F73EC0EF02FB406D0040191
:101EE000670E826F73EC0EF005D00401470E826F0F
:101EF00073EC0EF02FB606D00401740E826F73ECF3
:101F00000EF005D00401540E826F73EC0EF051EF09
:101F100026F00401410E826F73EC0EF00301835131
:101F2000310AD8B42DEF12F003018351320AD8B42C
:101F30005DEF11F003018351330AD8B4E6EF10F0DE
:101F400003018351340AD8B4D6EF0FF00301835153
:101F5000350AD8B4B3EF0FF004013F0E826F73EC73
:101F60000EF051EF26F004012C0E826F73EC0EF090
:101F700003018451300AD8B4C6EF0FF00301845135
:101F8000310AD8B4CEEF0FF01FEF11F08B9004019F
:101F9000300E826F73EC0EF0D4EF0FF08B800401E3
:101FA000310E826F73EC0EF051EF26F0CC0E21EC67
:101FB0000BF0E8CF0BF004012C0E826F73EC0EF0E7
:101FC00003018451310AD8B4FAEF0FF003018451B0
:101FD000300AD8B4FCEF0FF0030184514D0AD8B495
:101FE00006EF10F003018451540AD8B40DEF10F03D
:101FF00024EF10F08A8401D08A940BAE04D00BAC8D
:1020000002D00BBA21D0E00E0B1218D01F0E0B1607
:102010008539E844E00B0B1211D0E00E0B1670EC82
:102020002DF085C332F186C333F10101296B7DECBC
:102030002DF0F4EC2CF000511F0B0B12CC0E0C6E9B
:102040000BC00BF00AEC0BF00401340E826F73EC42
:102050000EF004012C0E826F73EC0EF0CC0E21EC0E
:102060000BF0E8CF1AF08AB406D00401300E826F6C
:1020700073EC0EF005D00401310E826F73EC0EF09C
:1020800004012C0E826F73EC0EF01A38E840070B37
:10209000E8CF82F40401300E822773EC0EF00401C5
:1020A0002C0E826F73EC0EF02FEC2DF01A501F0BDC
:1020B000E8CF00F1D2EC2CF032C182F40401300EF2
:1020C000822773EC0EF033C182F40401300E8227B4
:1020D00073EC0EF004012C0E826F73EC0EF02FECFB
:1020E0002DF02DC000F100AF0BD0FF0E016FFF0EE1
:1020F000026FFF0E036F04012D0E826F73EC0EF062
:10210000D2EC2CF031C182F40401300E822773EC42
:102110000EF032C182F40401300E822773EC0EF00F
:1021200033C182F40401300E822773EC0EF00401F7
:102130002C0E826F73EC0EF02FEC2DF02CC000F102
:10214000D2EC2CF031C182F40401300E822773EC02
:102150000EF032C182F40401300E822773EC0EF0CF
:1021600033C182F40401300E822773EC0EF00401B7
:102170002C0E826F73EC0EF02FEC2DF02EC000F1C0
:1021800000AF0BD0FF0E016FFF0E026FFF0E036F4B
:1021900004012D0E826F73EC0EF0D2EC2CF031C1E5
:1021A00082F40401300E822773EC0EF032C182F407
:1021B0000401300E822773EC0EF033C182F4040167
:1021C000300E822773EC0EF051EF26F0CB0E21EC8F
:1021D0000BF0E8CF0BF004012C0E826F73EC0EF0C5
:1021E00003018451450AD8B40AEF11F00301845168
:1021F000440AD8B40DEF11F003018451300AD8B469
:1022000010EF11F003018451310AD8B414EF11F02A
:102210001FEF11F00B9E19EF11F00B8E19EF11F05B
:10222000FC0E0B1619EF11F0FC0E0B160B8019EFBC
:1022300011F0CB0E0C6E0BC00BF00AEC0BF004018E
:10224000330E826F73EC0EF004012C0E826F73EC70
:102250000EF0CB0E21EC0BF0E8CF19F019BE38EFE1
:1022600011F00401450E826F73EC0EF03DEF11F09A
:102270000401440E826F73EC0EF004012C0E826F89
:1022800073EC0EF00401300E826F73EC0EF004015B
:102290002C0E826F73EC0EF019B056EF11F00401A2
:1022A000300E826F73EC0EF05BEF11F00401310E13
:1022B000826F73EC0EF051EF26F0CA0E21EC0BF09A
:1022C000E8CF0BF004012C0E826F73EC0EF00301CB
:1022D0008451450AD8B499EF11F003018451440A9E
:1022E000D8B49CEF11F0030184514D0AD8B4A5EF86
:1022F00011F003018451410AD8B49FEF11F003019A
:102300008451460AD8B4A2EF11F003018451560A51
:10231000D8B4ADEF11F003018451500AD8B4B8EF2E
:1023200011F003018451520AD8B4BBEF11F0C4EF8D
:1023300011F00B9EBEEF11F00B8EBEEF11F00B9C57
:10234000BEEF11F00B8CBEEF11F0FC0E0B1685C327
:10235000E8FF030B0B12BEEF11F0C70E0B1685C37F
:10236000E8FF070BE846E846E8460B12BEEF11F01F
:102370000B84BEEF11F00B94BEEF11F0CA0E0C6E81
:102380000BC00BF00AEC0BF0CA0E21EC0BF0E8CFFF
:1023900018F00401320E826F73EC0EF004012C0E63
:1023A000826F73EC0EF018BEDDEF11F00401450EE4
:1023B000826F73EC0EF0E2EF11F00401440E826FB5
:1023C00073EC0EF004012C0E826F73EC0EF018C04B
:1023D000E8FF030BE8CF82F40401300E822773EC90
:1023E0000EF004012C0E826F73EC0EF018BC00EF9F
:1023F00012F00401410E826F73EC0EF005EF12F043
:102400000401460E826F73EC0EF004012C0E826FF5
:1024100073EC0EF018C0E8FF380BE842E842E842DF
:10242000E8CF82F40401300E822773EC0EF0040131
:102430002C0E826F73EC0EF018B426EF12F004012C
:10244000520E826F73EC0EF02BEF12F00401500E5F
:10245000826F73EC0EF051EF26F0C90E21EC0BF0F9
:10246000E8CF0BF004012C0E826F73EC0EF0030129
:102470008451450AD8B44BEF12F003018451440A49
:10248000D8B44EEF12F0030184514D0AD8B451EF85
:1024900012F05FEF12F00B9E59EF12F00B8E59EF16
:1024A00012F0F80E0B1685C3E8FF070B0B1259EF5D
:1024B00012F0C90E0C6E0BC00BF00AEC0BF004010D
:1024C000310E826F73EC0EF004012C0E826F73ECF0
:1024D0000EF0C90E21EC0BF0E8CF17F017BE06D0B6
:1024E0000401450E826F73EC0EF005D00401440E1A
:1024F000826F73EC0EF004012C0E826F73EC0EF001
:1025000017C0E8FF070BE8CF82F40401300E8227E2
:1025100073EC0EF004012C0E826F73EC0EF007804A
:102520002FEC2DF028C0E8FF003B00430043030BD5
:10253000D2EC2CF033C182F40401300E822773EC0C
:102540000EF004012C0E826F73EC0EF02FEC2DF0C8
:1025500028C001F1019F019D29C000F10101D2ECC9
:102560002CF02FC182F40401300E822773EC0EF0A0
:1025700030C182F40401300E822773EC0EF031C1B9
:1025800082F40401300E822773EC0EF032C182F423
:102590000401300E822773EC0EF033C182F4040183
:1025A000300E822773EC0EF004012C0E826F73EC58
:1025B0000EF02FEC2DF02AC001F12BC000F1D890C5
:1025C00001330033D890013300330101D2EC2CF0F9
:1025D0002FC182F40401300E822773EC0EF030C15B
:1025E00082F40401300E822773EC0EF031C182F4C4
:1025F0000401300E822773EC0EF032C182F4040124
:10260000300E822773EC0EF033C182F40401300ED9
:10261000822773EC0EF051EF26F0FC0E21EC0BF04C
:10262000E8CF0BF003018351520AD8B444EF13F002
:1026300003018351720AD8B447EF13F003018351A9
:10264000500AD8B44AEF13F003018351700AD8B48A
:102650004DEF13F003018351550AD8B450EF13F036
:1026600003018351750AD8B453EF13F0030183516A
:10267000430AD8B45CEF13F003018351630AD8B462
:102680005FEF13F068EF13F00B9062EF13F00B8025
:1026900062EF13F00B9262EF13F00B8262EF13F014
:1026A0000B9462EF13F00B8462EF13F00B9662EF62
:1026B00013F00B8662EF13F00B9862EF13F00B88A8
:1026C00062EF13F0FC0E0C6E0BC00BF00AEC0BF07B
:1026D0000401590E826F73EC0EF011901192119457
:1026E0001198FC0E21EC0BF0E8CF0BF00BA0118041
:1026F0000BA211820BA411840BA8118811A088EFE2
:1027000013F00401520E826F73EC0EF08DEF13F094
:102710000401720E826F73EC0EF011A897EF13F0A4
:102720000401430E826F73EC0EF09CEF13F0040172
:10273000630E826F73EC0EF011A2A6EF13F004018A
:10274000500E826F73EC0EF0ABEF13F00401700EBD
:10275000826F73EC0EF011A4B5EF13F00401550E67
:10276000826F73EC0EF0BAEF13F00401750E826FF6
:1027700073EC0EF051EF26F004016D0E826F73ECD6
:102780000EF003018351300AD8B414EF14F00301A2
:102790008351310AD8B427EF14F003018351320A70
:1027A000D8B43AEF14F053EF26F004014D0E826FC7
:1027B00073EC0EF070EC2DF084C331F185C332F16F
:1027C00086C333F10101296B7DEC2DF0F4EC2CF084
:1027D00003018351300AD8B4FCEF13F00301835195
:1027E000310AD8B404EF14F003018351320AD8B48B
:1027F0000CEF14F053EF26F0FD0E0C6E00C10BF041
:102800000AEC0BF014EF14F0FE0E0C6E00C10BF08E
:102810000AEC0BF027EF14F0FF0E0C6E00C10BF06A
:102820000AEC0BF03AEF14F00401300E826F73ECF7
:102830000EF004012C0E826F73EC0EF02FEC2DF0D5
:10284000FD0E21EC0BF0E8CF00F14BEF14F004018A
:10285000310E826F73EC0EF004012C0E826F73EC5C
:102860000EF02FEC2DF0FE0E21EC0BF0E8CF00F176
:102870004BEF14F00401320E826F73EC0EF02FEC6C
:102880002DF004012C0E826F73EC0EF0FF0E21EC84
:102890000BF0E8CF00F1D2EC2CF031C182F404014E
:1028A000300E822773EC0EF032C182F40401300E38
:1028B000822773EC0EF033C182F40401300E8227BC
:1028C00073EC0EF051EF26F003018351300AD8B4B7
:1028D0005FEF19F003018351310AD8B48CEF1AF07D
:1028E00003018351320AD8B4FAEF1AF0030183517D
:1028F000330AD8B40AEF1BF003018351340AD8B469
:102900001AEF1BF003018351350AD8B4A0EF1CF075
:1029100003018351360AD8B4CEEF1CF00301835172
:10292000370AD8B437EF17F003018351380AD8B407
:10293000D5EF17F003018351460AD8B4F3EF1BF02B
:10294000030183514D0AD8B4B0EF15F00301835150
:102950006D0AD8B4CAEF15F0030183515A0AD8B4EE
:1029600006EF1AF003018351490AD8B4CEEF1DF0E7
:1029700003018351500AD8B400EF1DF003018351C5
:10298000540AD8B479EF1DF003018351630AD8B417
:10299000EAEF15F003018351430AD8B4E2EF16F0D1
:1029A00003018351730AD8B4E8EF15F00301835192
:1029B000610AD8B4FDEF14F003018351650AD8B45D
:1029C000AFEF19F003018351450AD8B4BDEF19F0F8
:1029D00003018351620AD8B4CBEF19F0030183518C
:1029E000420AD8B4D9EF19F003018351760AD8B45A
:1029F000E7EF19F0D8A453EF26F004014C0E826FD4
:102A000073EC0EF00401610E826F73EC0EF05FEC5C
:102A10002EF004012C0E826F73EC0EF02FEC2DF0D3
:102A2000AFC500F10101D2EC2CF031C182F40401F8
:102A3000300E822773EC0EF032C182F40401300EA6
:102A4000822773EC0EF033C182F40401300E82272A
:102A500073EC0EF004012C0E826F73EC0EF02FEC71
:102A60002DF0B0C500F10101D2EC2CF031C182F49F
:102A70000401300E822773EC0EF032C182F404019F
:102A8000300E822773EC0EF033C182F40401300E55
:102A9000822773EC0EF004012C0E826F73EC0EF0A3
:102AA0002FEC2DF0B1C500F10101D2EC2CF031C1B9
:102AB00082F40401300E822773EC0EF032C182F4EE
:102AC0000401300E822773EC0EF033C182F404014E
:102AD000300E822773EC0EF004012C0E826F73EC23
:102AE0000EF02FEC2DF0B2C500F10101D2EC2CF06C
:102AF00031C182F40401300E822773EC0EF032C132
:102B000082F40401300E822773EC0EF033C182F49C
:102B10000401300E822773EC0EF004012C0E826F3C
:102B200073EC0EF02FEC2DF0B6C500F10101D2ECE4
:102B30002CF031C182F40401300E822773EC0EF0C8
:102B400032C182F40401300E822773EC0EF033C1DF
:102B500082F40401300E822773EC0EF0FCEF1CF0BF
:102B600070EC2DF084C333F17DEC2DF0F4EC2CF0FF
:102B7000200E0C6E00C10BF00AEC0BF000C12FF51B
:102B800005012F51000A06E005012F51010A02E05C
:102B9000F9EC2EF004014C0E826F73EC0EF0040180
:102BA0004D0E826F73EC0EF004012C0E826F73ECED
:102BB0000EF02FEC2DF02FC500F1D2EC2CF033C12C
:102BC00082F40401300E822773EC0EF0FCEF1CF04F
:102BD000EFEF33F004014C0E826F73EC0EF0040142
:102BE000630E826F73EC0EF0B7EC2DF004012C0E27
:102BF000826F73EC0EF0FFEC15F0FCEF1CF02FEC85
:102C00002DF0B5C500F10101003B0F0E0017D2EC0D
:102C10002CF033C182F40401300E822773EC0EF0E5
:102C2000B5C500F101010F0E01010017D2EC2CF027
:102C300033C182F40401300E822773EC0EF00401DC
:102C40002D0E826F73EC0EF0B4C500F10101003B54
:102C50000F0E0017D2EC2CF033C182F40401300EB9
:102C6000822773EC0EF0B4C500F101010F0E0101D3
:102C70000017D2EC2CF033C182F40401300E82270D
:102C800073EC0EF004012D0E826F73EC0EF0B3C5E1
:102C900000F10101003B0F0E0017D2EC2CF033C104
:102CA00082F40401300E822773EC0EF0B3C500F1FC
:102CB00001010F0E01010017D2EC2CF033C182F498
:102CC0000401300E822773EC0EF00401200E826F97
:102CD00073EC0EF0B2C500F10F0E01010017D2EC3B
:102CE0002CF033C182F40401300E822773EC0EF015
:102CF0000401200E826F73EC0EF0B1C500F10101EA
:102D00000101003B0F0E0017D2EC2CF033C182F40E
:102D10000401300E822773EC0EF0B1C500F1010101
:102D20000F0E01010017D2EC2CF033C182F4040124
:102D3000300E822773EC0EF004013A0E826F73ECB2
:102D40000EF0B0C500F10101003B0F0E0017D2ECF0
:102D50002CF033C182F40401300E822773EC0EF0A4
:102D6000B0C500F101010F0E01010017D2EC2CF0EB
:102D700033C182F40401300E822773EC0EF004019B
:102D80003A0E826F73EC0EF0AFC500F10101003B0B
:102D90000F0E0017D2EC2CF033C182F40401300E78
:102DA000822773EC0EF0AFC500F101010F0E001782
:102DB000D2EC2CF033C182F40401300E822773EC84
:102DC0000EF0120084C3E8FF0F0BE83AE8CFB5F528
:102DD00085C3E8FF0F0B0501B51387C3E8FF0F0B91
:102DE000E83AE8CFB4F588C3E8FF0F0B0501B41348
:102DF0008AC3E8FF0F0BE83AE8CFB3F58BC3E8FFCF
:102E00000F0B0501B3138DC3E8FF0F0BE8CFB2F52D
:102E10008FC3E8FF0F0BE83AE8CFB1F590C3E8FFA6
:102E20000F0B0501B11392C3E8FF0F0BE83AE8CF8F
:102E3000B0F593C3E8FF0F0B0501B01395C3E8FF8E
:102E40000F0BE83AE8CFAFF596C3E8FF0F0B05018B
:102E5000AF1312EC2EF004014C0E826F73EC0EF0E7
:102E60000401430E826F73EC0EF0F4EF15F007844B
:102E700004014C0E826F73EC0EF00401370E826F6A
:102E800073EC0EF004012C0E826F73EC0EF0050152
:102E90002E51130A06E005012E51170A0DE0D2EF5C
:102EA00017F00101000E006F000E016F100E026F8F
:102EB000000E036F65EF17F00101000E006F000EAA
:102EC000016F000E026F010E036FD2EC2CF02AC1CD
:102ED00082F40401300E822773EC0EF02BC182F4D1
:102EE0000401300E822773EC0EF02CC182F4040131
:102EF000300E822773EC0EF02DC182F40401300EE7
:102F0000822773EC0EF02EC182F40401300E82276A
:102F100073EC0EF02FC182F40401300E822773ECA3
:102F20000EF030C182F40401300E822773EC0EF0F3
:102F300031C182F40401300E822773EC0EF032C1ED
:102F400082F40401300E822773EC0EF033C182F458
:102F50000401300E822773EC0EF004012C0E826FF8
:102F600073EC0EF00101100E006F000E016F000EE9
:102F7000026F000E036FD2EC2CF031C182F4040119
:102F8000300E822773EC0EF032C182F40401300E51
:102F9000822773EC0EF033C182F40401300E8227D5
:102FA00073EC0EF00794FCEF1CF00501216B226B13
:102FB000236B246B04014C0E826F73EC0EF0040142
:102FC000380E826F73EC0EF004012C0E826F73ECDE
:102FD0000EF00101100E006F000E016F000E026F67
:102FE000000E036FD2EC2CF02AC182F40401300EE3
:102FF000822773EC0EF02BC182F40401300E82277D
:1030000073EC0EF02CC182F40401300E822773ECB5
:103010000EF02DC182F40401300E822773EC0EF005
:103020002EC182F40401300E822773EC0EF02FC102
:1030300082F40401300E822773EC0EF030C182F46A
:103040000401300E822773EC0EF031C182F40401CA
:10305000300E822773EC0EF032C182F40401300E80
:10306000822773EC0EF033C182F40401300E822704
:1030700073EC0EF004012C0E826F73EC0EF025C57C
:1030800000F126C501F127C502F128C503F10101B0
:10309000100E046F000E056F000E066F000E076F16
:1030A00065EC2CF000C133F501C134F502C135F5F2
:1030B00003C136F5D2EC2CF02AC182F40401300EA3
:1030C000822773EC0EF02BC182F40401300E8227AC
:1030D00073EC0EF02CC182F40401300E822773ECE5
:1030E0000EF02DC182F40401300E822773EC0EF035
:1030F0002EC182F40401300E822773EC0EF02FC132
:1031000082F40401300E822773EC0EF030C182F499
:103110000401300E822773EC0EF031C182F40401F9
:10312000300E822773EC0EF032C182F40401300EAF
:10313000822773EC0EF033C182F40401300E822733
:1031400073EC0EF07DEC0EF005013367AFEF18F075
:103150003467AFEF18F03567AFEF18F0366702D07D
:103160004EEF19F0129E129C21C500F122C501F10B
:1031700023C502F124C503F1899A400EC76E200EC3
:10318000C66E9E96C69E0B0EC96EFF0E9EB602D0F0
:10319000E82EFCD79E96C69E02C1C9FFFF0E9EB6C2
:1031A00002D0E82EFCD79E96C69E01C1C9FFFF0E35
:1031B0009EB602D0E82EFCD79E96C69E00C1C9FFDF
:1031C000FF0E9EB602D0E82EFCD79E96C69EC95230
:1031D000FF0E9EB602D0E82EFCD70501100E326F0E
:1031E000040114EE00F080517F0BE1269E96C69EEE
:1031F000C952FF0E9EB602D0E82EFCD7C9CFE7FF1A
:103200000401802B0501322FF0EF18F0898A33C5B5
:1032100000F134C501F135C502F136C503F10101F4
:10322000010E046F000E056F000E066F000E076F93
:1032300034EC2CF000C133F501C134F502C135F591
:1032400003C136F5050133672DEF19F034672DEF13
:1032500019F035672DEF19F0366702D04EEF19F0EF
:1032600021C500F122C501F123C502F124C503F1F6
:103270000101100E046F000E056F000E066F000EA8
:10328000076F39EC2CF000C121F501C122F502C114
:1032900023F503C124F5128E53EF26F00401450EE9
:1032A000826F73EC0EF004014F0E826F73EC0EF020
:1032B0000401460E826F73EC0EF0FCEF1CF00784E5
:1032C000B0EC33F02FEC2DF02DC500F1D2EC2CF04A
:1032D00004014C0E826F73EC0EF00401300E826F0D
:1032E00073EC0EF004012C0E826F73EC0EF031C102
:1032F00082F40401300E822773EC0EF032C182F4A6
:103300000401300E822773EC0EF033C182F4040105
:10331000300E822773EC0EF004012C0E826F73ECDA
:103320000EF02FEC2DF02EC500F1D2EC2CF031C1B7
:1033300082F40401300E822773EC0EF032C182F465
:103340000401300E822773EC0EF033C182F40401C5
:10335000300E822773EC0EF00794FCEF1CF0040192
:103360004C0E826F73EC0EF00401650E826F73ECED
:103370000EF0D5EC2FF0FCEF1CF004014C0E826F28
:1033800073EC0EF00401450E826F73EC0EF0ECEC62
:103390002FF0FCEF1CF004014C0E826F73EC0EF06A
:1033A0000401620E826F73EC0EF01AEC30F0FCEF49
:1033B0001CF004014C0E826F73EC0EF00401420EFF
:1033C000826F73EC0EF003EC30F0FCEF1CF00401A4
:1033D0004C0E826F73EC0EF00401760E826F73EC6C
:1033E0000EF004012C0E826F73EC0EF010A807D0C3
:1033F0000401310E826F73EC0EF0FCEF1CF004013F
:10340000300E826F73EC0EF0FCEF1CF004014C0EDA
:10341000826F73EC0EF004015A0E826F73EC0EF0A3
:1034200004012C0E826F73EC0EF0B0EC33F02FEC35
:103430002DF005012E51130A06E005012E51170A41
:103440000DE037EF1AF00101000E006F000E016F62
:10345000100E026F000E036F37EF1AF00101000E1D
:10346000006F000E016F000E026F010E036F01016D
:10347000100E046F000E056F000E066F000E076F32
:1034800065EC2CF0D2EC2CF02AC182F40401300E51
:10349000822773EC0EF02BC182F40401300E8227D8
:1034A00073EC0EF02CC182F40401300E822773EC11
:1034B0000EF02DC182F40401300E822773EC0EF061
:1034C0002EC182F40401300E822773EC0EF02FC15E
:1034D00082F40401300E822773EC0EF030C182F4C6
:1034E0000401300E822773EC0EF031C182F4040126
:1034F000300E822773EC0EF032C182F40401300EDC
:10350000822773EC0EF033C182F40401300E82275F
:1035100073EC0EF0FCEF1CF0078404014C0E826F7C
:1035200073EC0EF00401310E826F73EC0EF00401A7
:103530002C0E826F73EC0EF025C500F126C501F14B
:1035400027C502F128C503F10101100E046F000E1A
:10355000056F000E066F000E076F65EC2CF0D2ECC5
:103560002CF02AC182F40401300E822773EC0EF095
:103570002BC182F40401300E822773EC0EF02CC1B3
:1035800082F40401300E822773EC0EF02DC182F418
:103590000401300E822773EC0EF02EC182F4040178
:1035A000300E822773EC0EF02FC182F40401300E2E
:1035B000822773EC0EF030C182F40401300E8227B2
:1035C00073EC0EF031C182F40401300E822773ECEB
:1035D0000EF032C182F40401300E822773EC0EF03B
:1035E00033C182F40401300E822773EC0EF007948D
:1035F000FCEF1CF0078404014C0E826F73EC0EF09C
:103600000401320E826F73EC0EF008EC32F0079476
:10361000FCEF1CF0078404014C0E826F73EC0EF07B
:103620000401330E826F73EC0EF065EC32F00794F8
:1036300097EF1AF0078404014C0E826F73EC0EF0C2
:103640000401340E826F73EC0EF004012C0E826FB5
:1036500073EC0EF070EC2DF084C32AF185C32BF1CE
:1036600086C32CF187C32DF188C32EF189C32FF1B6
:103670008AC330F18BC331F18CC332F18DC333F186
:103680000101296B7DEC2DF0F4EC2CF0100E046F91
:10369000000E056F000E066F000E076F45EC2CF054
:1036A00000C121F501C122F502C123F503C124F5B2
:1036B00063EC33F038C5AFF539C5B0F53AC5B1F5AF
:1036C0003BC5B2F53CC5B3F53DC5B4F53EC5B5F552
:1036D000FFEC15F004012C0E826F73EC0EF03FC569
:1036E00000F140C501F141C502F142C503F10101FC
:1036F000000E046F000E056F010E066F000E076FBF
:1037000065EC2CF0D2EC2CF0296789EF1BF08EEFE2
:103710001BF004012D0E826F73EC0EF030C182F4A9
:103720000401300E822773EC0EF031C182F40401E3
:10373000300E822773EC0EF004012E0E826F73ECB4
:103740000EF032C182F40401300E822773EC0EF0C9
:1037500033C182F40401300E822773EC0EF00401B1
:103760002C0E826F73EC0EF02FEC2DF043C500F1A0
:1037700044C501F17DEC27F004012C0E826F73EC3F
:103780000EF02FEC2DF045C500F1D2EC2CF031C13C
:1037900082F40401300E822773EC0EF032C182F401
:1037A0000401300E822773EC0EF033C182F4040161
:1037B000300E822773EC0EF004012C0E826F73EC36
:1037C0000EF037C5E8FFE8B806D00401300E826F6E
:1037D00073EC0EF005D00401310E826F73EC0EF025
:1037E0000794FCEF1CF070EC2DF085C32AF186C322
:1037F0002BF187C32CF188C32DF189C32EF18AC325
:103800002FF18BC330F18CC331F18DC332F18EC3F4
:1038100033F10101296B7DEC2DF0F4EC2CF001016A
:10382000010E046F000E056F000E066F000E076F8D
:1038300034EC2CF0100E046F000E056F000E066FB6
:10384000000E076F45EC2CF000C129F501C12AF5E7
:1038500002C12BF503C12CF58FEC31F004014C0EA5
:10386000826F73EC0EF00401460E826F73EC0EF063
:1038700004012C0E826F73EC0EF025C500F126C5F5
:1038800001F127C502F128C503F10101100E046FF3
:10389000000E056F000E066F000E076F65EC2CF032
:1038A000D2EC2CF02AC182F40401300E822773EC92
:1038B0000EF02BC182F40401300E822773EC0EF05F
:1038C0002CC182F40401300E822773EC0EF02DC15E
:1038D00082F40401300E822773EC0EF02EC182F4C4
:1038E0000401300E822773EC0EF02FC182F4040124
:1038F000300E822773EC0EF030C182F40401300EDA
:10390000822773EC0EF031C182F40401300E82275D
:1039100073EC0EF032C182F40401300E822773EC96
:103920000EF033C182F40401300E822773EC0EF0E6
:10393000FCEF1CF00F9865EC32F0308053EF26F06E
:1039400004014C0E826F73EC0EF00401350E826F91
:1039500073EC0EF004012C0E826F73EC0EF02FEC62
:103960002DF00784B9C500F10794D2EC2CF031C1D9
:1039700082F40401300E822773EC0EF032C182F41F
:103980000401300E822773EC0EF033C182F404017F
:10399000300E822773EC0EF0FCEF1CF028EC32F0B6
:1039A0002FEC2DF037C500F1D2EC2CF004014C0EB9
:1039B000826F73EC0EF00401360E826F73EC0EF022
:1039C00004012C0E826F73EC0EF031C182F40401FD
:1039D000300E822773EC0EF032C182F40401300EF7
:1039E000822773EC0EF033C182F40401300E82277B
:1039F00073EC0EF0FCEF1CF07DEC0EF053EF26F0B4
:103A000004014C0E826F73EC0EF00401500E826FB5
:103A100073EC0EF004012C0E826F73EC0EF085C374
:103A20002AF186C32BF187C32CF188C32DF189C3FA
:103A30002EF18AC32FF18BC330F18CC331F18DC3CA
:103A400032F18EC333F101017DEC2DF0F4EC2CF05A
:103A500003018451530A0DE0030184514D0A38E0FB
:103A60000401780E826F73EC0EF07DEC0EF053EFD4
:103A700026F00401530E826F73EC0EF0250E0C6ECF
:103A800000C10BF00AEC0BF0260E0C6E01C10BF01E
:103A90000AEC0BF0270E0C6E02C10BF00AEC0BF0D7
:103AA000280E0C6E03C10BF00AEC0BF000C157F5A9
:103AB00001C158F502C159F503C15AF500C15BF5C2
:103AC00001C15CF502C15DF503C15EF5DDEF1DF0DE
:103AD00004014D0E826F73EC0EF0290E0C6E00C1C6
:103AE0000BF00AEC0BF000C15FF500C160F5DDEFF3
:103AF0001DF004014C0E826F73EC0EF00401540EA5
:103B0000826F73EC0EF004012C0E826F73EC0EF0DA
:103B100084C32AF185C32BF186C32CF187C32DF111
:103B200088C32EF189C32FF18AC330F18BC331F1E1
:103B30008DC332F18EC333F101017DEC2DF0F4EC35
:103B40002CF00101000E046F000E056F010E066FD0
:103B5000000E076F45EC2CF0210E0C6E00C10BF02F
:103B60000AEC0BF0220E0C6E01C10BF00AEC0BF00C
:103B7000230E0C6E02C10BF00AEC0BF0240E0C6E3F
:103B800003C10BF00AEC0BF000C161F501C162F555
:103B900002C163F503C164F5DDEF1DF004014C0EB5
:103BA000826F73EC0EF00401490E826F73EC0EF01D
:103BB00004012C0E826F73EC0EF0250E21EC0BF03D
:103BC000E8CF00F1260E21EC0BF0E8CF01F1270E33
:103BD00021EC0BF0E8CF02F1280E21EC0BF0E8CF3E
:103BE00003F1D2EC2CF095EC2AF00401730E826FF5
:103BF00073EC0EF004012C0E826F73EC0EF02FECC0
:103C00002DF0290E21EC0BF0E8CF00F1D2EC2CF0D6
:103C100095EC2AF004016D0E826F73EC0EF0040136
:103C20002C0E826F73EC0EF05BC500F15CC501F1E8
:103C30005DC502F15EC503F1D2EC2CF095EC2AF0E3
:103C40000401730E826F73EC0EF004012C0E826F70
:103C500073EC0EF02FEC2DF060C500F1D2EC2CF0DF
:103C600095EC2AF004016D0E826F73EC0EF00401E6
:103C70002C0E826F73EC0EF061C500F162C501F18C
:103C800063C502F164C503F16EEC26F004012C0E4D
:103C9000826F73EC0EF07DEC0EF053EF26F083C3D1
:103CA0002AF184C32BF185C32CF186C32DF187C380
:103CB0002EF188C32FF189C330F18AC331F18BC350
:103CC00032F18CC333F101017DEC2DF0F4EC2CF0DA
:103CD000160E0C6E00C10BF00AEC0BF0170E0C6EFA
:103CE00001C10BF00AEC0BF0180E0C6E02C10BF0C8
:103CF0000AEC0BF0190E0C6E03C10BF00AEC0BF082
:103D000000C18AF101C18BF102C18CF103C18DF1B7
:103D100000C18EF101C18FF102C190F103C191F197
:103D200031EF1FF083C32AF184C32BF185C32CF13B
:103D300086C32DF187C32EF188C32FF189C330F1DB
:103D40008AC331F18BC332F18CC333F101017DECB5
:103D50002DF0F4EC2CF000C18AF101C18BF102C10D
:103D60008CF103C18DF100C18EF101C18FF102C14F
:103D700090F103C191F131EF1FF083C32AF184C3A5
:103D80002BF185C32CF186C32DF187C32EF188C397
:103D90002FF189C330F18AC331F18CC332F18DC365
:103DA00033F101017DEC2DF0F4EC2CF00101000E5B
:103DB000046F000E056F010E066F000E076F45ECD5
:103DC0002CF01A0E0C6E00C10BF00AEC0BF01B0E5F
:103DD0000C6E01C10BF00AEC0BF01C0E0C6E02C154
:103DE0000BF00AEC0BF01D0E0C6E03C10BF00AEC8D
:103DF0000BF000C192F101C193F102C194F103C132
:103E000095F131EF1FF083C32AF184C32BF185C3F1
:103E10002CF186C32DF187C32EF188C32FF189C3FE
:103E200030F18AC331F18CC332F18DC333F101011A
:103E30007DEC2DF0F4EC2CF00101000E046F000E6F
:103E4000056F010E066F000E076F45EC2CF000C1E8
:103E500092F101C193F102C194F103C195F131EFE7
:103E60001FF0160E21EC0BF0E8CF00F1170E21EC3D
:103E70000BF0E8CF01F1180E21EC0BF0E8CF02F1C6
:103E8000190E21EC0BF0E8CF03F1D2EC2CF095ECFD
:103E90002AF00401730E826F73EC0EF004012C0EF5
:103EA000826F73EC0EF08AC100F18BC101F18CC1FD
:103EB00002F18DC103F1D2EC2CF095EC2AF0040153
:103EC000730E826F73EC0EF004012C0E826F73EC94
:103ED0000EF01A0E21EC0BF0E8CF00F11B0E21ECD6
:103EE0000BF0E8CF01F11C0E21EC0BF0E8CF02F152
:103EF0001D0E21EC0BF0E8CF03F16EEC26F004016F
:103F00002C0E826F73EC0EF092C100F193C101F19F
:103F100094C102F195C103F16EEC26F07DEC0EF038
:103F200053EF26F00401690E826F73EC0EF004016A
:103F30002C0E826F73EC0EF00101040E006F000E68
:103F4000016F000E026F000E036FD2EC2CF02CC13B
:103F500082F40401300E822773EC0EF02DC182F43E
:103F60000401300E822773EC0EF02EC182F404019E
:103F7000300E822773EC0EF02FC182F40401300E54
:103F8000822773EC0EF030C182F40401300E8227D8
:103F900073EC0EF031C182F40401300E822773EC11
:103FA0000EF032C182F40401300E822773EC0EF061
:103FB00033C182F40401300E822773EC0EF0040149
:103FC0002C0E826F73EC0EF00101060E006F000ED6
:103FD000016F000E026F000E036FD2EC2CF02CC1AB
:103FE00082F40401300E822773EC0EF02DC182F4AE
:103FF0000401300E822773EC0EF02EC182F404010E
:10400000300E822773EC0EF02FC182F40401300EC3
:10401000822773EC0EF030C182F40401300E822747
:1040200073EC0EF031C182F40401300E822773EC80
:104030000EF032C182F40401300E822773EC0EF0D0
:1040400033C182F40401300E822773EC0EF00401B8
:104050002C0E826F73EC0EF00101320E006F000E19
:10406000016F000E026F000E036FD2EC2CF02CC11A
:1040700082F40401300E822773EC0EF02DC182F41D
:104080000401300E822773EC0EF02EC182F404017D
:10409000300E822773EC0EF02FC182F40401300E33
:1040A000822773EC0EF030C182F40401300E8227B7
:1040B00073EC0EF031C182F40401300E822773ECF0
:1040C0000EF032C182F40401300E822773EC0EF040
:1040D00033C182F40401300E822773EC0EF0040128
:1040E0002C0E826F73EC0EF0200EF86EF76AF66AF3
:1040F00004010900F5CF82F473EC0EF00900F5CF4E
:1041000082F473EC0EF00900F5CF82F473EC0EF03C
:104110000900F5CF82F473EC0EF00900F5CF82F4BC
:1041200073EC0EF00900F5CF82F473EC0EF0090089
:10413000F5CF82F473EC0EF00900F5CF82F473EC46
:104140000EF07DEC0EF053EF26F08351630AD8A4F5
:1041500051EF26F08451610AD8A451EF26F0855121
:104160006C0AD8A451EF26F08651410A3FE08651EF
:10417000440A1BE08651420AD8B409EF21F0865167
:10418000350AD8B4DDEF27F08651360AD8B432EFBD
:1041900028F08651370AD8B49BEF28F08651380AA8
:1041A000D8B4F9EF28F051EF26F00798079A0401E8
:1041B0007A0E826F73EC0EF00401780E826F73EC4E
:1041C0000EF00401640E826F73EC0EF00401550EC4
:1041D000826F73EC0EF0F2EF20F004014C0E826F50
:1041E00073EC0EF07DEC0EF053EF26F00788079A83
:1041F00004017A0E826F73EC0EF00401410E826F9F
:1042000073EC0EF00401610E826F73EC0EF0E6EFBA
:1042100020F00798078A04017A0E826F73EC0EF083
:104220000401420E826F73EC0EF00401610E826F86
:1042300073EC0EF0E6EF20F00101666727EF21F046
:10424000676727EF21F0686727EF21F0696715D0CE
:104250004F6732EF21F0506732EF21F0516732EFB4
:1042600021F052670AD00101000E006F000E016FAD
:10427000000E026F000E036F120011B80AD0010188
:10428000620E046F010E056F000E066F000E076FC1
:1042900009D00101A70E046F020E056F000E066F14
:1042A000000E076F66C100F167C101F168C102F13C
:1042B00069C103F134EC2CF003BFCFEF21F0119A68
:1042C000119C0101000E046FA80E056F550E066FBC
:1042D000020E076F66C100F167C101F168C102F10A
:1042E00069C103F166C186F167C187F168C188F1D0
:1042F00069C189F134EC2CF003BF0BD00101000E31
:10430000866FA80E876F550E886F020E896F118A0F
:10431000119C0E0E21EC0BF0E8CF18F10F0E21ECE2
:104320000BF0E8CF19F1100E21EC0BF0E8CF1AF1E9
:10433000110E21EC0BF0E8CF1BF17DEC2BF086C1C8
:1043400004F187C105F188C106F189C107F134EC98
:104350002CF0078241EC2BF07DEC2BF0079241EC26
:104360002BF086C100F187C101F188C102F189C13A
:1043700003F1079241EC2BF0CC0E046FE00E056FB9
:10438000870E066F050E076F34EC2CF000C118F194
:1043900001C119F102C11AF103C11BF13BD0119CFB
:1043A000119A0101800E006F1A0E016F060E026F46
:1043B000000E036F4FC104F150C105F151C106F168
:1043C00052C107F134EC2CF003AF05D02FEC2DF0E7
:1043D000118C119A12000E0E21EC0BF0E8CF18F19F
:1043E0000F0E21EC0BF0E8CF19F1100E21EC0BF0C1
:1043F000E8CF1AF1110E21EC0BF0E8CF1BF14FC101
:1044000000F150C101F151C102F152C103F1078223
:1044100041EC2BF018C100F119C101F11AC102F1F0
:104420001BC103F112000401730E826F73EC0EF0D6
:1044300004012C0E826F73EC0EF0078462C166F1EA
:1044400063C167F164C168F165C169F14BC14FF1A6
:104450004CC150F14DC151F14EC152F157C159F10A
:1044600058C15AF1079439EC22F07DEC0EF053EF6D
:1044700026F066C100F167C101F168C102F169C1AE
:1044800003F10101D2EC2CF095EC2AF00401630E4B
:10449000826F73EC0EF004012C0E826F73EC0EF041
:1044A0004FC100F150C101F151C102F152C103F1FC
:1044B0000101D2EC2CF095EC2AF00401660E826F1B
:1044C00073EC0EF004012C0E826F73EC0EF02FECE7
:1044D0002DF059C100F15AC101F10101D2EC2CF0CB
:1044E00095EC2AF00401740E826F73EC0EF012004A
:1044F00010820401530E826F73EC0EF004012C0E37
:10450000826F73EC0EF083C32AF184C32BF185C351
:104510002CF186C32DF187C32EF188C32FF189C3F7
:1045200030F18AC331F18BC332F18CC333F1010115
:104530007DEC2DF0F4EC2CF000C166F101C167F1C7
:1045400002C168F103C169F18EC32AF18FC32BF157
:1045500090C32CF191C32DF192C32EF193C32FF18F
:1045600094C330F195C331F196C332F197C333F15F
:1045700001017DEC2DF0F4EC2CF000C14FF101C1F4
:1045800050F102C151F103C152F170EC2DF099C309
:104590002FF19AC330F19BC331F19CC332F19DC31B
:1045A00033F101017DEC2DF0F4EC2CF000C159F158
:1045B00001C15AF139EC22F004012C0E826F73EC28
:1045C0000EF0F2EF22F0118E19A002D019AE108C6D
:1045D00018BE02D018A4108E8251520A02E10F8236
:1045E00001D00F928251750A02E1108401D010941B
:1045F0008251550A02E1108601D0109611A003D015
:1046000011A401D01084078410B260EF23F010A42D
:104610004CEF23F0B6C166F1B7C167F1B8C168F1DC
:10462000B9C169F1BAC16AF1BBC16BF1BCC16CF12E
:10463000BDC16DF1BEC16EF1BFC16FF1C0C170F1FE
:10464000C1C171F1C2C172F1C3C173F1C4C174F1CE
:10465000C5C175F1C6C176F1C7C177F1C8C178F19E
:10466000C9C179F1CAC17AF1CBC17BF1CCC17CF16E
:10467000CDC17DF1CEC17EF1CFC17FF1D0C180F13E
:10468000D1C181F1D2C182F1D3C183F1D4C184F10E
:10469000D5C185F154EF23F062C166F163C167F1C2
:1046A00064C168F165C169F14BC14FF14CC150F172
:1046B0004DC151F14EC152F157C159F158C15AF192
:1046C00007940FA082EF23F0010192676FEF23F0B0
:1046D00093676FEF23F094676FEF23F0956773EFA5
:1046E00023F082EF23F01CEC21F092C104F193C17E
:1046F00005F194C106F195C107F134EC2CF003BF2C
:1047000019EF26F01CEC21F00101000E046F000EE1
:10471000056F010E066F000E076F65EC2CF011A0FF
:104720002CD011A22AD0D2EC2CF0296701D007D0CE
:1047300004012D0E826F73EC0EF017EF26F030C1DE
:1047400082F40401300E822773EC0EF031C182F442
:104750000401300E822773EC0EF032C182F40401A2
:10476000300E822773EC0EF033C182F40401300E58
:10477000822773EC0EF017EF26F012A8C5D012981E
:104780001AC01BF01B3A1B42070E1B1600011B50E0
:10479000000AD8B450EF24F000011B50010AD8B42D
:1047A000DCEF23F000011B50020AD8B4DAEF23F04B
:1047B00082EF24F082EF24F02FEC2DF02AC001F1DB
:1047C0002BC000F1D89001330033D890013300336F
:1047D0000101630E046F000E056F000E066F000EE0
:1047E000076F65EC2CF0280E046F000E056F000EAD
:1047F000066F000E076F34EC2CF000C12DF02FEC8B
:104800002DF028C001F1019F019D29C000F1010197
:10481000A40E046F000E056F000E066F000E076FEA
:1048200065EC2CF000C12CF000C104F101C105F1D0
:1048300002C106F103C107F1640E006F000E016FA3
:10484000000E026F000E036F34EC2CF0050E046FA7
:10485000000E056F000E066F000E076F65EC2CF062
:1048600000C104F101C105F102C106F103C107F164
:104870002FEC2DF02DC000F134EC2CF000C12EF007
:104880002EC0E8FF050F2D5C03E78A8482EF24F039
:104890002EC0E8FF0A0F2D5C01E68A9482EF24F017
:1048A00000C124F101C125F102C126F103C127F1A4
:1048B0002FEC2DF035EC2DF01A501F0BE8CF00F146
:1048C0000101640E046F000E056F000E066F000EEE
:1048D000076F45EC2CF024C104F125C105F126C178
:1048E00006F127C107F134EC2CF003BF02D08A9403
:1048F00001D08A8424C100F125C101F126C102F151
:1049000027C103F119EF26F000C124F101C125F1FF
:1049100002C126F103C127F110AE4CD0109E00C198
:1049200008F101C109F102C10AF103C10BF1D2EC96
:104930002CF030C1D6F131C1D7F132C1D8F133C139
:10494000D9F108C100F109C101F10AC102F10BC19D
:1049500003F101016C0E046F070E056F000E066F68
:10496000000E076F34EC2CF003BF04D00101550E8C
:10497000DA6F1CD008C100F109C101F10AC102F1CE
:104980000BC103F10101A40E046F060E056F000EAA
:10499000066F000E076F34EC2CF003BF04D001014A
:1049A0007F0EDA6F03D00101FF0EDA6F1C8E11AE9D
:1049B00019EF26F024C100F125C101F126C102F151
:1049C00027C103F110A4ECEF24F00401750E826FEF
:1049D00073EC0EF0F1EF24F00401720E826F73ECB1
:1049E0000EF004012C0E826F73EC0EF0D2EC2CF062
:1049F000296700EF25F00401200E826F03EF25F0F8
:104A000004012D0E826F73EC0EF030C182F40401AC
:104A1000300E822773EC0EF031C182F40401300EA7
:104A2000822773EC0EF004012E0E826F73EC0EF0F1
:104A300032C182F40401300E822773EC0EF033C1D0
:104A400082F40401300E822773EC0EF004016D0E27
:104A5000826F73EC0EF004012C0E826F73EC0EF07B
:104A60004FC100F150C101F151C102F152C103F136
:104A70000101D2EC2CF095EC2AF00401480E826F73
:104A800073EC0EF004017A0E826F73EC0EF00401E9
:104A90002C0E826F73EC0EF066C100F167C101F15C
:104AA00068C102F169C103F10101D2EC2CF095EC6F
:104AB0002AF00401630E826F73EC0EF004012C0ED9
:104AC000826F73EC0EF066C100F167C101F168C13D
:104AD00002F169C103F101010A0E046F000E056FB6
:104AE000000E066F000E076F45EC2CF0000E046FF1
:104AF000120E056F000E066F000E076F65EC2CF0AE
:104B0000D2EC2CF02AC182F40401300E822773EC1F
:104B10000EF02BC182F40401300E822773EC0EF0EC
:104B20002CC182F40401300E822773EC0EF02DC1EB
:104B300082F40401300E822773EC0EF02EC182F451
:104B40000401300E822773EC0EF02FC182F40401B1
:104B5000300E822773EC0EF030C182F40401300E67
:104B6000822773EC0EF004012E0E826F73EC0EF0B0
:104B700031C182F40401300E822773EC0EF032C191
:104B800082F40401300E822773EC0EF033C182F4FC
:104B90000401300E822773EC0EF00401730E826F55
:104BA00073EC0EF004012C0E826F73EC0EF02FEC00
:104BB0002DF059C100F15AC101F17DEC27F00FB27F
:104BC000E5EF25F00FA017EF26F004012C0E826F01
:104BD00073EC0EF0200EF86EF76AF66A0401090015
:104BE000F5CF82F473EC0EF00900F5CF82F473EC8C
:104BF0000EF00900F5CF82F473EC0EF00900F5CF4A
:104C000082F473EC0EF00900F5CF82F473EC0EF031
:104C10000900F5CF82F473EC0EF00900F5CF82F4B1
:104C200073EC0EF00900F5CF82F473EC0EF07DEC1E
:104C30000EF00F9053EF26F00401630E826F73ECB9
:104C40000EF004012C0E826F73EC0EF059EC26F07E
:104C500004012C0E826F73EC0EF0CCEC26F00401F4
:104C60002C0E826F73EC0EF048EC27F004012C0E32
:104C7000826F73EC0EF00101F80E006FCD0E016F24
:104C8000660E026F030E036F6EEC26F004012C0E0D
:104C9000826F73EC0EF05EEC27F07DEC0EF053EFBC
:104CA00026F07DEC0EF00301C26B0790109262EFCC
:104CB00029F0D8900E0E21EC0BF0E8CF00F10F0E8A
:104CC00021EC0BF0E8CF01F1100E21EC0BF0E8CF56
:104CD00002F1110E21EC0BF0E8CF03F10101000EFF
:104CE000046F000E056F010E066F000E076F65EC76
:104CF0002CF0D2EC2CF02AC182F40401300E822771
:104D000073EC0EF02BC182F40401300E822773EC99
:104D10000EF02CC182F40401300E822773EC0EF0E9
:104D20002DC182F40401300E822773EC0EF02EC1E7
:104D300082F40401300E822773EC0EF02FC182F44E
:104D40000401300E822773EC0EF030C182F40401AE
:104D5000300E822773EC0EF031C182F40401300E64
:104D6000822773EC0EF004012E0E826F73EC0EF0AE
:104D700032C182F40401300E822773EC0EF033C18D
:104D800082F40401300E822773EC0EF004016D0EE4
:104D9000826F73EC0EF01200120E21EC0BF0E8CFD4
:104DA00000F1130E21EC0BF0E8CF01F1140E21EC11
:104DB0000BF0E8CF02F1150E21EC0BF0E8CF03F178
:104DC00001010A0E046F000E056F000E066F000E43
:104DD000076F45EC2CF0000E046F120E056F000EED
:104DE000066F000E076F65EC2CF0D2EC2CF02AC198
:104DF00082F40401300E822773EC0EF02BC182F492
:104E00000401300E822773EC0EF02CC182F40401F1
:104E1000300E822773EC0EF02DC182F40401300EA7
:104E2000822773EC0EF02EC182F40401300E82272B
:104E300073EC0EF02FC182F40401300E822773EC64
:104E40000EF030C182F40401300E822773EC0EF0B4
:104E500004012E0E826F73EC0EF031C182F4040156
:104E6000300E822773EC0EF032C182F40401300E52
:104E7000822773EC0EF033C182F40401300E8227D6
:104E800073EC0EF00401730E826F73EC0EF01200DF
:104E90000A0E21EC0BF0E8CF00F10B0E21EC0BF029
:104EA000E8CF01F10C0E21EC0BF0E8CF02F10D0E72
:104EB00021EC0BF0E8CF03F17DEF27F0060E21EC9B
:104EC0000BF0E8CF00F1070E21EC0BF0E8CF01F179
:104ED000080E21EC0BF0E8CF02F1090E21EC0BF0EB
:104EE000E8CF03F17DEF27F001012FEC2DF00784CF
:104EF00057C100F158C101F107940101E80E046F98
:104F0000800E056F000E066F000E076F45EC2CF04B
:104F1000000E046F040E056F000E066F000E076F83
:104F200065EC2CF0880E046F130E056F000E066FF3
:104F3000000E076F34EC2CF00A0E046F000E056FA4
:104F4000000E066F000E076F65EC2CF0D2EC2CF013
:104F500001012967B1EF27F00401200E826FB4EF41
:104F600027F004012D0E826F73EC0EF030C182F435
:104F70000401300E822773EC0EF031C182F404017B
:104F8000300E822773EC0EF032C182F40401300E31
:104F9000822773EC0EF004012E0E826F73EC0EF07C
:104FA00033C182F40401300E822773EC0EF0040149
:104FB000430E826F73EC0EF0120087C32AF188C390
:104FC0002BF189C32CF18AC32DF18BC32EF18CC335
:104FD0002FF18DC330F18EC331F190C332F191C303
:104FE00033F10101296B7DEC2DF0F4EC2CF0010183
:104FF000000E046F000E056F010E066F000E076FA6
:1050000045EC2CF00E0E0C6E00C10BF00AEC0BF010
:105010000F0E0C6E01C10BF00AEC0BF0100E0C6EB3
:1050200002C10BF00AEC0BF0110E0C6E03C10BF079
:105030000AEC0BF004017A0E826F73EC0EF004019F
:105040002C0E826F73EC0EF00401350E826F73EC40
:105050000EF004012C0E826F73EC0EF059EC26F06A
:10506000F2EF20F087C32AF188C32BF189C32CF11A
:105070008AC32DF18BC32EF18CC32FF18DC330F178
:105080008EC331F190C332F191C333F10101296B29
:105090007DEC2DF0F4EC2CF0880E046F130E056FF0
:1050A000000E066F000E076F39EC2CF0000E046F37
:1050B000040E056F000E066F000E076F45EC2CF016
:1050C0000101E80E046F800E056F000E066F000EE2
:1050D000076F65EC2CF00A0E0C6E00C10BF00AECA9
:1050E0000BF00B0E0C6E01C10BF00AEC0BF00C0E6A
:1050F0000C6E02C10BF00AEC0BF00D0E0C6E03C12E
:105100000BF00AEC0BF004017A0E826F73EC0EF0D8
:1051100004012C0E826F73EC0EF00401360E826FC8
:1051200073EC0EF004012C0E826F73EC0EF048EC61
:1051300027F0F2EF20F087C32AF188C32BF189C34F
:105140002CF18AC32DF18BC32EF18CC32FF18DC3AB
:1051500030F18FC331F190C332F191C333F10101CA
:105160007DEC2DF0F4EC2CF0000E046F120E056FA8
:10517000000E066F000E076F45EC2CF001010A0EC1
:10518000046F000E056F000E066F000E076F65ECD2
:105190002CF0120E0C6E00C10BF00AEC0BF0130E8B
:1051A0000C6E01C10BF00AEC0BF0140E0C6E02C178
:1051B0000BF00AEC0BF0150E0C6E03C10BF00AECB1
:1051C0000BF004017A0E826F73EC0EF004012C0ECA
:1051D000826F73EC0EF00401370E826F73EC0EF0E9
:1051E00004012C0E826F73EC0EF0CCEC26F0F2EF83
:1051F00020F087C32AF188C32BF189C32CF18AC31D
:105200002DF18BC32EF18CC32FF18DC330F18EC3E2
:1052100031F190C332F191C333F10101296B7DEC7F
:105220002DF0F4EC2CF0880E046F130E056F000EB9
:10523000066F000E076F39EC2CF0000E046F040EA1
:10524000056F000E066F000E076F45EC2CF0010194
:10525000E80E046F800E056F000E066F000E076FDC
:1052600065EC2CF0060E0C6E00C10BF00AEC0BF096
:10527000070E0C6E01C10BF00AEC0BF0080E0C6E61
:1052800002C10BF00AEC0BF0090E0C6E03C10BF01F
:105290000AEC0BF004017A0E826F73EC0EF004013D
:1052A0002C0E826F73EC0EF00401380E826F73ECDB
:1052B0000EF004012C0E826F73EC0EF05EEC27F002
:1052C000F2EF20F007A8D5EF29F00101800E006F62
:1052D0001A0E016F060E026F000E036F4BC104F130
:1052E0004CC105F14DC106F14EC107F134EC2CF073
:1052F00003BF1BEF2AF08FEC2AF04BC100F14CC129
:1053000001F14DC102F14EC103F1078241EC2BF0D6
:1053100018C104F119C105F11AC106F11BC107F149
:10532000F80E006FCD0E016F660E026F030E036F55
:1053300034EC2CF00E0E0C6E00C10BF00AEC0BF0EE
:105340000F0E0C6E01C10BF00AEC0BF0100E0C6E80
:1053500002C10BF00AEC0BF0110E0C6E03C10BF046
:105360000AEC0BF0078401012FEC2DF057C100F17E
:1053700058C101F107940A0E0C6E00C10BF00AEC43
:105380000BF00B0E0C6E01C10BF00AEC0BF00C0EC7
:105390000C6E02C10BF00AEC0BF00D0E0C6E03C18B
:1053A0000BF00AEC0BF01BEF2AF007AA1BEF2AF018
:1053B000078401012FEC2DF057C100F158C101F114
:1053C0000794060E0C6E00C10BF00AEC0BF0070EF2
:1053D0000C6E01C10BF00AEC0BF0080E0C6E02C152
:1053E0000BF00AEC0BF0090E0C6E03C10BF00AEC8B
:1053F0000BF0078462C100F163C101F164C102F1E5
:1054000065C103F10794120E0C6E00C10BF00AEC9B
:105410000BF0130E0C6E01C10BF00AEC0BF0140E26
:105420000C6E02C10BF00AEC0BF0150E0C6E03C1F2
:105430000BF00AEC0BF00798079A040180518119D0
:105440007F0B0DE09EA8FED714EE00F081517F0B7C
:10545000E126E750812B0F01AD6E1DEF2AF005010B
:105460002F51010A13E081AA57EF2AF005012F51AD
:10547000000A0AE00FB846EF2AF00501306746EF50
:105480002AF00FB846EF2AF0EFEF33F081B857EF6C
:105490002AF05FEC2EF057EF2AF0602F57EF2AF03A
:1054A0005FC560F50501010E306F3C0E316FBAEF3C
:1054B0000DF018C100F119C101F11AC102F11BC1AF
:1054C00003F1000E046F000E056F010E066F000E53
:1054D000076F65EC2CF029A184EF2AF02051D8B495
:1054E00084EF2AF018C100F119C101F11AC102F1CB
:1054F0001BC103F1000E046F000E056F0A0E066F4C
:10550000000E076F65EC2CF012000101045100132E
:105510000551011306510213075103131200010133
:10552000186B196B1A6B1B6B12002AC182F40401F1
:10553000300E822773EC0EF02BC182F40401300E82
:10554000822773EC0EF02CC182F40401300E822706
:1055500073EC0EF02DC182F40401300E822773EC3F
:105560000EF02EC182F40401300E822773EC0EF08F
:105570002FC182F40401300E822773EC0EF030C18B
:1055800082F40401300E822773EC0EF031C182F4F4
:105590000401300E822773EC0EF032C182F4040154
:1055A000300E822773EC0EF033C182F40401300E0A
:1055B000822773EC0EF012002FC182F40401300E2A
:1055C000822773EC0EF030C182F40401300E822782
:1055D00073EC0EF031C182F40401300E822773ECBB
:1055E0000EF032C182F40401300E822773EC0EF00B
:1055F00033C182F40401300E822773EC0EF01200E6
:10560000060E1E6E060E1F6E060E206E1E2E06EF76
:105610002BF01F2E06EF2BF0202E06EF2BF08B84A5
:10562000020E1E6E020E1F6E020E206E1E2E16EF52
:105630002BF01F2E16EF2BF0202E16EF2BF08B9455
:105640001200FF0E1F6E1FC020F0030E1E6E8B8413
:105650001E2E27EF2BF0030E1E6E202E27EF2BF0B1
:105660008B941FC020F0030E1E6E1E2E35EF2BF004
:10567000030E1E6E203E35EF2BF01F2E23EF2BF076
:1056800012000101005305E1015303E1025301E15E
:10569000002B04EC2CF02FEC2DF03951006F3A5117
:1056A000016F420E046F4B0E056F000E066F000E69
:1056B000076F45EC2CF000C104F101C105F102C1F6
:1056C00006F103C107F118C100F119C101F11AC1B6
:1056D00002F11BC103F107B272EF2BF039EC2CF091
:1056E00074EF2BF034EC2CF000C118F101C119F16A
:1056F00002C11AF103C11BF112002FEC2DF059C1A8
:1057000000F15AC101F1060E21EC0BF0E8CF04F1D3
:10571000070E21EC0BF0E8CF05F1080E21EC0BF0A1
:10572000E8CF06F1090E21EC0BF0E8CF07F134ECDD
:105730002CF000C124F101C125F102C126F103C101
:1057400027F1290E046F000E056F000E066F000E84
:10575000076F45EC2CF0EE0E046F430E056F000E44
:10576000066F000E076F39EC2CF024C104F125C13F
:1057700005F126C106F127C107F145EC2CF000C167
:105780001CF101C11DF102C11EF103C11FF1120E76
:1057900021EC0BF0E8CF04F1130E21EC0BF0E8CF75
:1057A00005F1140E21EC0BF0E8CF06F1150E21ECFB
:1057B0000BF0E8CF07F10D0E006F000E016F000E29
:1057C000026F000E036F45EC2CF0180E046F000EF4
:1057D000056F000E066F000E076F65EC2CF01CC104
:1057E00004F11DC105F11EC106F11FC107F139EC1D
:1057F0002CF06A0E046F2A0E056F000E066F000E65
:10580000076F34EC2CF01200BF0EFA6E200E3A6FC8
:10581000396BD8900037013702370337D8B015EF0E
:105820002CF03A2F0AEF2CF039073A070353D8B47B
:1058300012000331070B80093F6F03390F0B010F73
:10584000396F80EC5FF0406F390580EC5FF0405DB0
:10585000405F396B3F33D8B0392739333FA92AEF3E
:105860002CF0405139271200010154EC2DF0D8B032
:105870001200010103510719346F17EC2DF0D89075
:105880000751031934AF800F12000101346B3BEC58
:105890002DF0D8A051EC2DF0D8B0120026EC2DF050
:1058A0002FEC2DF01F0E366F67EC2DF00B35D8B0B6
:1058B00017EC2DF0D8A00335D8B01200362F54EFD6
:1058C0002CF034B13EEC2DF012000101346B045188
:1058D0000511061107110008D8A03BEC2DF0D8A047
:1058E00051EC2DF0D8B01200086B096B0A6B0B6BF2
:1058F00067EC2DF01F0E366F67EC2DF007510B5D36
:10590000D8A48FEF2CF006510A5DD8A48FEF2CF0AD
:105910000551095DD8A48FEF2CF00451085DD8A083
:10592000A2EF2CF00451085F0551D8A0053D095F96
:105930000651D8A0063D0A5F0751D8A0073D0B5F6E
:10594000D8900081362F7CEF2CF034B13EEC2DF056
:10595000346B3BEC2DF0D8906BEC2DF007510B5DC8
:10596000D8A4BFEF2CF006510A5DD8A4BFEF2CF0ED
:105970000551095DD8A4BFEF2CF00451085DD8A0F3
:10598000CEEF2CF0003FCEEF2CF0013FCEEF2CF00D
:10599000023FCEEF2CF0032BD8B4120034B13EEC12
:1059A0002DF012000101346B3BEC2DF0D8B0120049
:1059B00070EC2DF0200E366F0037013702370337B9
:1059C00011EE33F00A0E376FE7360A0EE75CD8B0F7
:1059D000E76EE552372FE4EF2CF0362FDCEF2CF09A
:1059E00034B12981D890120001010A0E346F200EC3
:1059F000366F11EE29F03451376F0A0ED890E65207
:105A0000D8B0E726E732372FFFEF2CF0033302330D
:105A100001330033362FF9EF2CF0E750FF0FD8A0F9
:105A20000335D8B0120029B13EEC2DF0120004511C
:105A300000270551D8B0053D01270651D8B0063DD5
:105A400002270751D8B0073D032712000051086F05
:105A50000151096F02510A6F03510B6F12000101CE
:105A6000006B016B026B036B12000101046B056B91
:105A7000066B076B12000335D8A012000351800B90
:105A8000001F011F021F031F003F4EEF2DF0013FBB
:105A90004EEF2DF0023F4EEF2DF0032B342B03255C
:105AA00012000735D8A012000751800B041F051FF4
:105AB000061F071F043F64EF2DF0053F64EF2DF034
:105AC000063F64EF2DF0072B342B0725120000371B
:105AD000013702370337083709370A370B37120007
:105AE0000101296B2A6B2B6B2C6B2D6B2E6B2F6B93
:105AF000306B316B326B336B120001012A510F0B8B
:105B00002A6F2B510F0B2B6F2C510F0B2C6F2D511C
:105B10000F0B2D6F2E510F0B2E6F2F510F0B2F6F61
:105B200030510F0B306F31510F0B316F32510F0B62
:105B3000326F33510F0B336F120010A806D08994C7
:105B4000000EC76E220EC66E05D08984000EC76E89
:105B5000220EC66E050EE82EFED7120010A802D047
:105B6000898401D08994050EE82EFED712009DECA1
:105B70002DF09E96C69E000EC96EFF0E9EB602D0F8
:105B8000E82EFCD79E96C69E000EC96EFF0E9EB6EE
:105B900002D0E82EFCD7C9CFAFF59E96C69E000E68
:105BA000C96EFF0E9EB602D0E82EFCD7C9CFB0F565
:105BB0009E96C69E000EC96EFF0E9EB602D0E82EBF
:105BC000FCD7C9CFB1F59E96C69E000EC96EFF0EDA
:105BD0009EB602D0E82EFCD7C9CFB2F59E96C69EDF
:105BE000000EC96EFF0E9EB602D0E82EFCD7C9CFBC
:105BF000B3F59E96C69E000EC96EFF0E9EB602D0ED
:105C0000E82EFCD7C9CFB4F59E96C69E000EC96E8D
:105C1000FF0E9EB602D0E82EFCD7C9CFB5F5AEEC8C
:105C20002DF012009DEC2DF09E96C69E800EC96E42
:105C3000FF0E9EB602D0E82EFCD79E96C69EAFC53C
:105C4000C9FFFF0E9EB602D0E82EFCD79E96C69ED8
:105C5000B0C5C9FFFF0E9EB602D0E82EFCD79E96B7
:105C6000C69EB1C5C9FFFF0E9EB602D0E82EFCD776
:105C70009E96C69EB2C5C9FFFF0E9EB602D0E82E04
:105C8000FCD79E96C69EB3C5C9FFFF0E9EB602D036
:105C9000E82EFCD79E96C69EB4C5C9FFFF0E9EB6E1
:105CA00002D0E82EFCD79E96C69EB5C5C9FFFF0E52
:105CB0009EB602D0E82EFCD7AEEC2DF012009DEC83
:105CC0002DF09E96C69E070EC96EFF0E9EB602D0A0
:105CD000E82EFCD79E96C69E000EC96EFF0E9EB69D
:105CE00002D0E82EFCD7C9CFAFF59E96C69E000E17
:105CF000C96EFF0E9EB602D0E82EFCD7C9CFB0F514
:105D00009E96C69E000EC96EFF0E9EB602D0E82E6D
:105D1000FCD7C9CFB1F59E96C69E000EC96EFF0E88
:105D20009EB602D0E82EFCD7C9CFB2F5AEEC2DF06E
:105D30009DEC2DF09E96C69E22C0C9FFFF0E9EB61A
:105D400002D0E82EFCD79E96C69E000EC96EFF0EAE
:105D50009EB602D0E82EFCD7C9CFB6F5AEEC2DF03A
:105D600012009DEC2DF09E96C69E870EC96EFF0E0A
:105D70009EB602D0E82EFCD79E96C69EAFC5C9FF40
:105D8000FF0E9EB602D0E82EFCD79E96C69EB0C5EA
:105D9000C9FFFF0E9EB602D0E82EFCD79E96C69E87
:105DA000B1C5C9FFFF0E9EB602D0E82EFCD79E9665
:105DB000C69EB2C5C9FFFF0E9EB602D0E82EFCD724
:105DC000AEEC2DF09DEC2DF09E96C69E23C0C9FF33
:105DD000FF0E9EB602D0E82EFCD79E96C69EB6C594
:105DE000C9FFFF0E9EB602D0E82EFCD7AEEC2DF018
:105DF00012009DEC2DF09E96C69E870EC96EFF0E7A
:105E00009EB602D0E82EFCD79E96C69E000EC96EA6
:105E1000FF0E9EB602D0E82EFCD79E96C69E800E40
:105E2000C96EFF0E9EB602D0E82EFCD79E96C69E87
:105E3000800EC96EFF0E9EB602D0E82EFCD79E964D
:105E4000C69E800EC96EFF0E9EB602D0E82EFCD70D
:105E5000AEEC2DF012009DEC2DF09E96C69E870EA6
:105E6000C96EFF0E9EB602D0E82EFCD79E96C69E47
:105E7000000EC96EFF0E9EB602D0E82EFCD79E968D
:105E8000C69E000EC96EFF0E9EB602D0E82EFCD74D
:105E90009E96C69E800EC96EFF0E9EB602D0E82E5C
:105EA000FCD79E96C69E800EC96EFF0E9EB602D08F
:105EB000E82EFCD7AEEC2DF0120010A817D09DEC08
:105EC0002DF09E96C69E8F0EC96EFF0E9EB602D016
:105ED000E82EFCD79E96C69E000EC96EFF0E9EB69B
:105EE00002D0E82EFCD7AEEC2DF012005FEC2EF0C5
:105EF000120010A82DD09DEC2DF09E96C69E23C0BA
:105F0000C9FFFF0E9EB602D0E82EFCD79E96C69E15
:105F1000450EC96EFF0E9EB602D0E82EFCD7AEEC41
:105F20002DF09DEC2DF09E96C69E8F0EC96EFF0E35
:105F30009EB602D0E82EFCD79E96C69E000EC96E75
:105F4000FF0E9EB602D0E82EFCD7AEEC2DF012006C
:105F50009DEC2DF09E96C69E23C0C9FFFF0E9EB6F7
:105F600002D0E82EFCD79E96C69E010EC96EFF0E8B
:105F70009EB602D0E82EFCD7AEEC2DF09DEC2DF0B5
:105F80009E96C69E910EC96EFF0E9EB602D0E82E5A
:105F9000FCD79E96C69EA50EC96EFF0E9EB602D079
:105FA000E82EFCD7AEEC2DF012009DEC2DF09E9665
:105FB000C69E23C0C9FFFF0E9EB602D0E82EFCD7B6
:105FC0009E96C69E810EC96EFF0E9EB602D0E82E2A
:105FD000FCD7AEEC2DF012009DEC2DF09E96C69EE7
:105FE00023C0C9FFFF0E9EB602D0E82EFCD79E96B6
:105FF000C69E010EC96EFF0E9EB602D0E82EFCD7DB
:10600000AEEC2DF012009DEC2DF09E96C69E910EEA
:10601000C96EFF0E9EB602D0E82EFCD79E96C69E95
:10602000A50EC96EFF0E9EB602D0E82EFCD7AEECD0
:106030002DF012009DEC2DF09E96C69E910EC96E1D
:10604000FF0E9EB602D0E82EFCD79E96C69E000E8E
:10605000C96EFF0E9EB602D0E82EFCD7AEEC2DF036
:1060600012000501256B266B276B286B899A400E61
:10607000C76E200EC66E9E96C69E030EC96EFF0E9C
:106080009EB602D0E82EFCD79E96C69E27C5C9FFB5
:10609000FF0E9EB602D0E82EFCD79E96C69E26C561
:1060A000C9FFFF0E9EB602D0E82EFCD79E96C69E74
:1060B00025C5C9FFFF0E9EB602D0E82EFCD79E96DE
:1060C000C69EC952FF0E9EB602D0E82EFCD7898A22
:1060D0000F01C950FF0A01E1120005012E51130AF8
:1060E00005E005012E51170A0CE012000501F00E23
:1060F000256FFF0E266F0F0E276F000E286F8AEF99
:1061000030F00501F00E256FFF0E266FFF0E276F92
:10611000000E286F899A400EC76E200EC66E9E969E
:10612000C69E030EC96EFF0E9EB602D0E82EFCD7A7
:106130009E96C69E27C5C9FFFF0E9EB602D0E82ECA
:10614000FCD79E96C69E26C5C9FFFF0E9EB602D0FE
:10615000E82EFCD79E96C69E25C5C9FFFF0E9EB6AB
:1061600002D0E82EFCD79E96C69EC952FF0E9EB660
:1061700002D0E82EFCD7898A0F01C950FF0A1DE022
:1061800005012E51130A05E005012E51170A0BE0F7
:1061900012000501000E256F000E266F100E276FEE
:1061A000000E286F12000501000E256F000E266FED
:1061B000000E276F010E286F12000501256B266B5C
:1061C000276B286B05012E51130A05E005012E519E
:1061D000170A0CE012000501000E216F000E226F5D
:1061E000080E236F000E246FFFEF30F00501000E44
:1061F000216F000E226F800E236F000E246F21C5C9
:1062000000F122C501F123C502F124C503F125C522
:1062100004F126C505F127C506F128C507F185EC6F
:106220002AF000C125F501C126F502C127F503C1F9
:1062300028F5899A400EC76E200EC66E9E96C69EA1
:10624000030EC96EFF0E9EB602D0E82EFCD79E96B6
:10625000C69E27C5C9FFFF0E9EB602D0E82EFCD70A
:106260009E96C69E26C5C9FFFF0E9EB602D0E82E9A
:10627000FCD79E96C69E25C5C9FFFF0E9EB602D0CE
:10628000E82EFCD79E96C69EC952FF0E9EB602D03F
:10629000E82EFCD7898AC950FF0A08E104C125F518
:1062A00005C126F506C127F507C128F5D8900501D7
:1062B00024332333223321332151F00B216F216703
:1062C00069EF31F0226769EF31F0236769EF31F050
:1062D0002467FFEF30F00501100E2527E86A26231A
:1062E000E86A2723E86A28231200E86A05012E518C
:1062F000130A06E005012E51170A0BE0020E1200E8
:1063000005012851000A03E12751F00B07E0010EB7
:10631000120005012851000A01E0010E120029C5F2
:1063200000F12AC501F12BC502F12CC503F125C5E9
:1063300004F126C505F127C506F128C507F134EC9F
:106340002CF003BF120075EC31F0D8A407EF32F047
:10635000899A400EC76E200EC66E9E96C69E060E89
:10636000C96EFF0E9EB602D0E82EFCD7898A899AA4
:106370009E96C69E020EC96EFF0E9EB602D0E82EF5
:10638000FCD79E96C69E27C5C9FFFF0E9EB602D0BB
:10639000E82EFCD79E96C69E26C5C9FFFF0E9EB668
:1063A00002D0E82EFCD79E96C69E25C5C9FFFF0EDB
:1063B0009EB602D0E82EFCD79E96C69E000EC96EF1
:1063C000FF0E9EB602D0E82EFCD7898A899A9E9647
:1063D000C69E050EC96EFF0E9EB602D0E82EFCD7F3
:1063E0009E96C69EC952FF0E9EB602D0E82EFCD7DE
:1063F000C9B0F0EF31F0898A0501100E2527E86A4F
:106400002623E86A2723E86A28238FEF31F0120059
:10641000899A400EC76E200EC66E9E96C69E060EC8
:10642000C96EFF0E9EB602D0E82EFCD7898A899AE3
:106430009E96C69EC70EC96EFF0E9EB602D0E82E6F
:10644000FCD7898A0501256B266B276B286B120008
:10645000899A400EC76E200EC66E9E96C69E050E89
:10646000C96EFF0E9EB602D0E82EFCD79E96C69E41
:10647000C952FF0E9EB602D0E82EFCD7C9CF37F521
:10648000898A1200899A400EC76E200EC66E9E96AB
:10649000C69EB90EC96EFF0E9EB602D0E82EFCD77E
:1064A000898A1200899A400EC76E200EC66E9E968B
:1064B000C69EAB0EC96EFF0E9EB602D0E82EFCD76C
:1064C000898AFF0EE82EFED7120075EC31F0D8A4B1
:1064D0001200899A400EC76E200EC66E9E96C69E0A
:1064E000030EC96EFF0E9EB602D0E82EFCD79E9614
:1064F000C69E27C5C9FFFF0E9EB602D0E82EFCD768
:106500009E96C69E26C5C9FFFF0E9EB602D0E82EF7
:10651000FCD79E96C69E25C5C9FFFF0E9EB602D02B
:10652000E82EFCD79E96C69EC952FF0E9EB602D09C
:10653000E82EFCD7898A0F01C950FF0AD8A462EF60
:1065400033F00501FE0E376F30A03799B7EC2DF010
:10655000AFC538F5B0C539F5B1C53AF5B2C53BF5AB
:10656000B3C53CF5B4C53DF5B5C53EF50784B6C128
:1065700066F1B7C167F1B8C168F1B9C169F14BC142
:106580004FF14CC150F14DC151F14EC152F157C1C3
:1065900059F158C15AF11CEC21F000C13FF501C17D
:1065A00040F502C141F503C142F505016167E0EF25
:1065B00032F06267E0EF32F06367E0EF32F0646779
:1065C000E4EF32F0F1EF32F061C504F162C505F19C
:1065D00063C506F164C507F134EC2CF003BF62EF2C
:1065E00033F059C143F55AC144F5B9C545F5BAC5AB
:1065F00046F507940501110E326F899A400EC76E59
:10660000200EC66E9E96C69E060EC96EFF0E9EB6E4
:1066100002D0E82EFCD7898A899A9E96C69E020EE1
:10662000C96EFF0E9EB602D0E82EFCD79E96C69E7F
:1066300027C5C9FFFF0E9EB602D0E82EFCD79E9656
:10664000C69E26C5C9FFFF0E9EB602D0E82EFCD717
:106650009E96C69E25C5C9FFFF0E9EB602D0E82EA7
:10666000FCD725EE37F0322F02D042EF33F09E9662
:10667000C69EDECFC9FFFF0E9EB602D0E82EFCD725
:1066800033EF33F0898A899A9E96C69E050EC96EAD
:10669000FF0E9EB602D0E82EFCD79E96C69EC9522B
:1066A000FF0E9EB602D0E82EFCD7C9B04DEF33F0F6
:1066B000898A0501100E2527E86A2623E86A272320
:1066C000E86A2823120021C500F122C501F123C583
:1066D00002F124C503F1899A400EC76E200EC66EE2
:1066E0009E96C69E0B0EC96EFF0E9EB602D0E82E79
:1066F000FCD79E96C69E02C1C9FFFF0E9EB602D071
:10670000E82EFCD79E96C69E01C1C9FFFF0E9EB61D
:1067100002D0E82EFCD79E96C69E00C1C9FFFF0E90
:106720009EB602D0E82EFCD79E96C69EC952FF0E9A
:106730009EB602D0E82EFCD725EE37F00501100EEC
:10674000326F9E96C69EC952FF0E9EB602D0E82EAC
:10675000FCD7C9CFDEFF322FA1EF33F0898A1200B8
:10676000899A400EC76E200EC66E9E96C69E900EEB
:10677000C96EFF0E9EB602D0E82EFCD79E96C69E2E
:10678000000EC96EFF0E9EB602D0E82EFCD79E9674
:10679000C69E000EC96EFF0E9EB602D0E82EFCD734
:1067A0009E96C69E000EC96EFF0E9EB602D0E82EC3
:1067B000FCD79E96C69EC952FF0E9EB602D0E82E0A
:1067C000FCD7C9CF2DF59E96C69EC952FF0E9EB628
:1067D00002D0E82EFCD7C9CF2EF5898A120000EC32
:1067E0002BF0B9C5E8FFD70802E300EC2BF0B9C5E0
:1067F000E8FFC80802E300EC2BF0B9C5E8FFB908D0
:1068000002E300EC2BF0B9C5E8FFAA0802E300ECB4
:106810002BF0B9C5E8FF9B0802E300EC2BF042EC3B
:1068200032F0F29CF29E8B94C69AC2909482948C21
:10683000720ED36ED3A4FED789968A909390F29A63
:10684000F2949D909E909D929E92F298F2925DECB1
:106850002FF0FF0EE8CF00F0E82EFED7002EFCD779
:10686000F290F286815081A838EF34F0F29E030056
:10687000F296F290010E306E038021EC2BF056EF71
:026880000BF01B
:10BF0000E844F926000C160C2B0C3F0C520C640C68
:10BF1000760C860C960CA50CB30CC10CCF0CDC0C6B
:06BF2000E80CF40C000C1B
:0200000400F00A
:0100C800FE39
:00000001FF
